:020000040000FA
:0408000098EF0BF072
:1008100003B275EF05F0F2B493EF05F09EB09BEFD5
:1008200005F09EB2A3EF05F0F2A81AEF04F0F2B2C1
:1008300023EF04F0F2B01FEF04F047EF0BF0F29655
:10084000F29047EF0BF0CD90F2929EA02DEF04F0C6
:100850000101533F2DEF04F0542BB2C1B6F1B3C1E7
:10086000B7F1B4C1B8F1B5C1B9F1AEC1B2F1AFC120
:10087000B3F1B0C1B4F1B1C1B5F1AAC1AEF1ABC130
:10088000AFF1ACC1B0F1ADC1B1F1A6C1AAF1A7C140
:10089000ABF1A8C1ACF1A9C1ADF1A2C1A6F1A3C150
:1008A000A7F1A4C1A8F1A5C1A9F19EC1A2F19FC160
:1008B000A3F1A0C1A4F1A1C1A5F19AC19EF19BC170
:1008C0009FF19CC1A0F19DC1A1F1CECF9AF1CFCFF4
:1008D0009BF153C19CF154C19DF1CF6ACE6A0101D5
:1008E000536B546B9E90CD800FBC0F8E0FBA7CEF74
:1008F00004F00F8A47EF0BF013880F8C0FBEB9EF8F
:1009000004F09AC19EF19BC19FF19CC1A0F19DC1D1
:10091000A1F19EC1A2F19FC1A3F1A0C1A4F1A1C107
:10092000A5F1A2C1A6F1A3C1A7F1A4C1A8F1A5C1D7
:10093000A9F1A6C1AAF1A7C1ABF1A8C1ACF1A9C1A7
:10094000ADF1AAC1AEF1ABC1AFF1ACC1B0F1ADC177
:10095000B1F1AEC1B2F1AFC1B3F1B0C1B4F1B1C147
:10096000B5F1B2C1B6F1B3C1B7F1B4C1B8F1B5C117
:10097000B9F101015E6B5F6B606B616B9A515E2731
:100980009B515F239C5160239D5161239E515E27A3
:100990009F515F23A0516023A1516123A2515E2783
:1009A000A3515F23A4516023A5516123A6515E2763
:1009B000A7515F23A8516023A9516123AA515E2743
:1009C000AB515F23AC516023AD516123AE515E2723
:1009D000AF515F23B0516023B1516123B2515E2703
:1009E000B3515F23B4516023B5516123B6515E27E3
:1009F000B7515F23B8516023B9516123D8900101E9
:100A0000613360335F335E33D8900101613360330B
:100A10005F335E33D8900101613360335F335E33FF
:100A200000C10CF101C10DF102C10EF103C10FF1C2
:100A300004C110F105C111F106C112F107C113F192
:100A400008C114F109C115F10AC116F10BC117F162
:100A500034C135F111B838EF05F00101620E046FB1
:100A6000010E056F000E066F000E076F41EF05F0D7
:100A70000101A70E046F020E056F000E066F000E37
:100A8000076F5EC100F15FC101F160C102F161C198
:100A900003F1CBEC30F003BF04D01CBE02D01CA08D
:100AA000108C11A059EF05F010BA59EF05F00F8026
:100AB000108A0CC100F10DC101F10EC102F10FC18C
:100AC00003F110C104F111C105F112C106F113C106
:100AD00007F114C108F115C109F116C10AF117C1D6
:100AE0000BF135C134F147EF0BF00392ABB2AB9889
:100AF000AB88030103EE00F080517F0BE92604C0B0
:100B0000EFFF802B8151805D700BD8A48B82000099
:100B10008051815D700BD8A48B9281518019D8B41B
:100B2000079047EF0BF0F2940101453F47EF0BF0C0
:100B3000462B47EF0BF09E900101533F47EF0BF020
:100B4000542B47EF0BF09E9211B843EF08F00400CE
:100B500066A1ABEF05F08BB4B5EF05F010ACB5EFC7
:100B600005F08B84109CB6EF05F08B94077C07ACE6
:100B7000D1EF05F0C274C2B4CBEF05F0C3CFB7F527
:100B8000C4CFB8F50501D890B833B733D890B8338F
:100B9000B733D2EF05F0C3CF55F1C4CF56F1D2EF42
:100BA00005F0C28207B444EF06F047C14BF148C1DB
:100BB0004CF149C14DF14AC14EF15EC162F15FC1D4
:100BC00063F160C164F161C165F113A8EAEF05F05A
:100BD000138C13989AC1BAF19BC1BBF19CC1BCF1B3
:100BE0009DC1BDF19EC1BEF19FC1BFF1A0C1C0F1C9
:100BF000A1C1C1F1A2C1C2F1A3C1C3F1A4C1C4F199
:100C0000A5C1C5F1A6C1C6F1A7C1C7F1A8C1C8F168
:100C1000A9C1C9F1AAC1CAF1ABC1CBF1ACC1CCF138
:100C2000ADC1CDF1AEC1CEF1AFC1CFF1B0C1D0F108
:100C3000B1C1D1F1B2C1D2F1B3C1D3F1B4C1D4F1D8
:100C4000B5C1D5F1B6C1D6F1B7C1D7F1B8C1D8F1A8
:100C5000B9C1D9F1B7C5B9F5B8C5BAF5B9C5BBF5CC
:100C6000BAC5BCF5010155515B2756515C23E86AB2
:100C70005D230E2E44EF06F05CC157F15DC158F1C3
:100C80005B6B5C6B5D6B078E0201002F47EF0BF017
:100C90003C0E006F1D50E00BE00AE86612881BBE98
:100CA00002D01BB4108E00C10CF101C10DF102C1C4
:100CB0000EF103C10FF104C110F105C111F106C11C
:100CC00012F107C113F108C114F109C115F10AC1EC
:100CD00016F10BC117F134C135F181AAACEF06F062
:100CE00015A4F7EF06F005012F51000AD8B43AEF2A
:100CF00007F005012F51010AD8B4B6EF06F005013F
:100D00002F51020AD8B4F7EF06F005012F51030A5C
:100D1000D8B4F7EF06F005012F51040AD8B4F7EF65
:100D200006F005012F51050AD8B4F7EF06F00501CA
:100D30002F51060AD8B4F7EF06F005012F51070A24
:100D4000D8B4F7EF06F005012F51320AD8B4B4EF4A
:100D500006F02F6B3AEF07F000011650030AD8B4E3
:100D6000F7EF06F03AEF07F03AEF07F005015767A3
:100D7000C1EF06F05867C1EF06F05967C1EF06F002
:100D80005A67C5EF06F03AEF07F05BC500F15CC5A6
:100D900001F15DC502F15EC503F10101010E046FB1
:100DA000000E056F000E066F000E076FCBEC30F0E3
:100DB00000C15BF501C15CF502C15DF503C15EF5E3
:100DC00001010067EBEF06F00167EBEF06F0026749
:100DD000EBEF06F003673AEF07F057C55BF558C530
:100DE0005CF559C55DF55AC55EF524EF07F00FBEF9
:100DF0000CEF07F010A011EF07F00101476708EFB3
:100E000007F0486708EF07F0496708EF07F04A67FF
:100E10000CEF07F011EF07F007AE11EF07F024EF2A
:100E200007F00501312F3AEF07F03C0E316F302FFC
:100E30003AEF07F00101000E626FE00E636FA50E3E
:100E4000646F010E656F138800011650000AD8B454
:100E500032EF07F000011650030AD8B437EF07F05D
:100E60003AEF07F00001010E166E3AEF07F00001AD
:100E7000040E166E0501666B37B740EF07F066810A
:100E80000CC100F10DC101F10EC102F10FC103F15E
:100E900010C104F111C105F112C106F113C107F12E
:100EA00014C108F115C109F116C10AF117C10BF1FE
:100EB00035C134F100C10CF101C10DF102C10EF1D7
:100EC00003C10FF104C110F105C111F106C112F106
:100ED00007C113F108C114F109C115F10AC116F1D6
:100EE0000BC117F134C135F101018E677FEF07F0B7
:100EF0008F677FEF07F090677FEF07F0916783EFD1
:100F000007F0B4EF07F092C100F193C101F194C171
:100F100002F195C103F10101010E046F000E056F8E
:100F2000000E066F000E076FCBEC30F000C192F19F
:100F300001C193F102C194F103C195F10101006770
:100F4000A9EF07F00167A9EF07F00267A9EF07F023
:100F50000367B4EF07F08EC192F18FC193F190C196
:100F600094F191C195F10F80D57ED5BE6ED0D6CFCC
:100F700047F1D7CF48F145C149F1E86AE8CF4AF1D6
:100F8000138A1CBE02D01CA0108C109047C100F127
:100F900048C101F149C102F14AC103F101010A0E40
:100FA000046F000E056F000E066F000E076FCBEC8E
:100FB00030F003AF1080010154A7EBEF07F00F9A58
:100FC0000F9C0F9E0101000E5E6F600E5F6F3D0E65
:100FD000606F080E616F010147BFFBEF07F04867C4
:100FE000FBEF07F04967FBEF07F04A67FBEF07F0FD
:100FF000F28820EF08F0F2985E6B5F6B606B616BBC
:101000009A6B9B6B9C6B9D6B9E6B9F6BA06BA16B9C
:10101000A26BA36BA46BA56BA66BA76BA86BA96B4C
:10102000AA6BAB6BAC6BAD6BAE6BAF6BB06BB16BFC
:10103000B26BB36BB46BB56BB66BB76BB86BB96BAC
:10104000D76AD66A0101456B466B0CC100F10DC130
:1010500001F10EC102F10FC103F110C104F111C180
:1010600005F112C106F113C107F114C108F115C150
:1010700009F116C10AF117C10BF135C134F147EF7F
:101080000BF047EF0BF00201002FABEF0AF0D59EFB
:10109000D6CF47F1D7CF48F145C149F1E86AE8CF4B
:1010A0004AF1138AD76AD66A0101456B466BD58E21
:1010B0001D50E00BE00AE86612881BBE02D01BB48C
:1010C000108E1AAE1F8C00C10CF101C10DF102C1CE
:1010D0000EF103C10FF104C110F105C111F106C1F8
:1010E00012F107C113F108C114F109C115F10AC1C8
:1010F00016F10BC117F134C135F10FA0109A11B8D8
:101100008DEF08F00101620E046F010E056F000EF5
:10111000066F000E076F96EF08F00101A70E046F2F
:10112000020E056F000E066F000E076F47C100F13B
:1011300048C101F149C102F14AC103F1CBEC30F0E1
:1011400003BFA9EF08F01CBE02D01CA0108C11B088
:101150000F800CC100F10DC101F10EC102F10FC1F0
:1011600003F110C104F111C105F112C106F113C15F
:1011700007F114C108F115C109F116C10AF117C12F
:101180000BF135C134F102013C0E006F00C10CF1CE
:1011900001C10DF102C10EF103C10FF104C110F143
:1011A00005C111F106C112F107C113F108C114F113
:1011B00009C115F10AC116F10BC117F134C135F19E
:1011C00081BAE6EF08F015B225EF09F015A025EF7A
:1011D00009F015A470EF09F005012F51000AD8B4E9
:1011E000B3EF09F005012F51010AD8B42FEF09F030
:1011F00005012F51020AD8B470EF09F005012F51F3
:10120000030AD8B470EF09F005012F51040AD8B4CD
:1012100070EF09F005012F51050AD8B470EF09F0FD
:1012200005012F51060AD8B470EF09F005012F51BE
:10123000070AD8B470EF09F005012F51320AD8B46B
:101240002DEF09F02F6BB3EF09F000011650030AE0
:10125000D8B470EF09F0B3EF09F0B3EF09F005016E
:1012600057673AEF09F058673AEF09F059673AEFD4
:1012700009F05A673EEF09F0B3EF09F05BC500F1E2
:101280005CC501F15DC502F15EC503F10101010E0E
:10129000046F000E056F000E066F000E076FCBEC9B
:1012A00030F000C15BF501C15CF502C15DF503C121
:1012B0005EF50101006764EF09F0016764EF09F072
:1012C000026764EF09F00367B3EF09F057C55BF5F8
:1012D00058C55CF559C55DF55AC55EF59DEF09F039
:1012E0000FBE85EF09F010A08AEF09F001014767F2
:1012F00081EF09F0486781EF09F0496781EF09F054
:101300004A6785EF09F08AEF09F007AE8AEF09F026
:101310009DEF09F00501312FB3EF09F03C0E316F5D
:10132000302FB3EF09F00101000E626FE00E636F22
:10133000A50E646F010E656F138800011650000A38
:10134000D8B4ABEF09F000011650030AD8B4B0EFDF
:1013500009F0B3EF09F00001010E166EB3EF09F0CA
:101360000001040E166E0501666B37B7B9EF09F080
:1013700066810CC100F10DC101F10EC102F10FC176
:1013800003F110C104F111C105F112C106F113C13D
:1013900007F114C108F115C109F116C10AF117C10D
:1013A0000BF135C134F100C10CF101C10DF102C1E5
:1013B0000EF103C10FF104C110F105C111F106C115
:1013C00012F107C113F108C114F109C115F10AC1E5
:1013D00016F10BC117F134C135F101018E67F8EF39
:1013E00009F08F67F8EF09F09067F8EF09F091675F
:1013F000FCEF09F02DEF0AF092C100F193C101F169
:1014000094C102F195C103F10101010E046F000EB8
:10141000056F000E066F000E076FCBEC30F000C1B9
:1014200092F101C193F102C194F103C195F101015F
:10143000006722EF0AF0016722EF0AF0026722EF4D
:101440000AF003672DEF0AF08EC192F18FC193F17C
:1014500090C194F191C195F10F80109047C100F1B6
:1014600048C101F149C102F14AC103F101010A0E6B
:10147000046F000E056F000E066F000E076FCBECB9
:1014800030F003AF1080010154A753EF0AF00F9A18
:101490000F9C0F9E0101000E5E6F600E5F6F3D0E90
:1014A000606F080E616F47C100F148C101F149C189
:1014B00002F14AC103F10101140E046F050E056F1C
:1014C000000E066F000E076FCBEC30F003AF6CEF31
:1014D0000AF0F28891EF0AF0F2985E6B5F6B606B36
:1014E000616B9A6B9B6B9C6B9D6B9E6B9F6BA06BF8
:1014F000A16BA26BA36BA46BA56BA66BA76BA86B70
:10150000A96BAA6BAB6BAC6BAD6BAE6BAF6BB06B1F
:10151000B16BB26BB36BB46BB56BB66BB76BB86BCF
:10152000B96B0CC100F10DC101F10EC102F10FC187
:1015300003F110C104F111C105F112C106F113C18B
:1015400007F114C108F115C109F116C10AF117C15B
:101550000BF135C134F104008BB4B6EF0AF010ACD6
:10156000B6EF0AF08B84109CB7EF0AF08B94077CDF
:1015700007ACD2EF0AF0C274C2B4CCEF0AF0C3CF0A
:10158000B7F5C4CFB8F50501D890B833B733D890C4
:10159000B833B733D3EF0AF0C3CF55F1C4CF56F108
:1015A000D3EF0AF0C28207B445EF0BF047C14BF10D
:1015B00048C14CF149C14DF14AC14EF15EC162F1E1
:1015C0005FC163F160C164F161C165F113A8EBEF24
:1015D0000AF0138C13989AC1BAF19BC1BBF19CC15C
:1015E000BCF19DC1BDF19EC1BEF19FC1BFF1A0C1C3
:1015F000C0F1A1C1C1F1A2C1C2F1A3C1C3F1A4C193
:10160000C4F1A5C1C5F1A6C1C6F1A7C1C7F1A8C162
:10161000C8F1A9C1C9F1AAC1CAF1ABC1CBF1ACC132
:10162000CCF1ADC1CDF1AEC1CEF1AFC1CFF1B0C102
:10163000D0F1B1C1D1F1B2C1D2F1B3C1D3F1B4C1D2
:10164000D4F1B5C1D5F1B6C1D6F1B7C1D7F1B8C1A2
:10165000D8F1B9C1D9F1B7C5B9F5B8C5BAF5B9C5A9
:10166000BBF5BAC5BCF5010155515B2756515C234A
:10167000E86A5D230E2E45EF0BF05CC157F15DC1AA
:1016800058F15B6B5C6B5D6B078E47EF0BF002C034
:10169000E0FF005001C0D8FF1000A6B24DEF0BF0E4
:1016A0000CC0A9FF0BC0A8FFA69EA69CA684F29E14
:1016B000550EA76EAA0EA76EA682F28EA694A6B2AB
:1016C0005FEF0BF00C2A1200A96EA69EA69CA680C6
:1016D000A8500C2A120004012C0E826FA2EC0EF00E
:1016E000E0EC31F00C5064EC0BF0E8CF00F10C5062
:1016F00064EC0BF0E8CF01F101AF84EF0BF00101D6
:10170000FF0E026FFF0E036F69EC31F0296790EF57
:101710000BF00401200E826FA2EC0EF095EF0BF09F
:1017200004012D0E826FA2EC0EF073EC2FF012006C
:1017300015941596076A0F6A106A116A126A136A7D
:10174000166A0F010D0EC16E860EC06E030EC26EBC
:101750000F01680E896E130E926E080E8A6EF30EDC
:10176000936E8B6A900E946EC80E64EC0BF0E8CF0B
:1017700025F000012550FE0AD8B4CAEF0BF0000195
:101780002550FD0AD8B4CFEF0BF00F0E266E8F0E4A
:10179000276E09D00E0E266E8E0E276E04D00D0E0B
:1017A000266E8D0E276E7EEC32F0BEEC33F0F18E9D
:1017B000F19EFC0E64EC0BF0E8CF0BF00BA0118057
:1017C0000BA211820BA411840BA81188C90E64EC22
:1017D0000BF0E8CF1AF0CA0E64EC0BF0E8CF1BF068
:1017E000CB0E64EC0BF0E8CF1CF0CC0E64EC0BF0ED
:1017F000E8CF1DF0FB0E64EC0BF0E8CF38F0CE0E16
:1018000064EC0BF0E8CF14F0CD0E64EC0BF0E8CFF5
:1018100037F01F6A206A0E6A01015B6B5C6B5D6BBF
:10182000576B586BF29A0101476B486B496B4A6BD7
:101830004B6B4C6B4D6B4E6B4F6B506B516B526BDC
:10184000456B466BD76AD66A0F01280ED56EF28AB1
:101850009D90B00ECD6E01015E6B5F6B606B616B36
:10186000626B636B646B656B666B676B686B696BF4
:10187000536B546BCF6ACE6A0F9A0F9C0F9E9D805C
:10188000760ECA6E9D8202013C0E006FCC6A160E67
:1018900064EC0BF0E8CF00F1170E64EC0BF0E8CF2E
:1018A00001F1180E64EC0BF0E8CF02F1190E64ECB4
:1018B0000BF0E8CF03F1010103AF79EF0CF0E0EC9E
:1018C00031F0160E0C6E00C10BF04DEC0BF0170E44
:1018D0000C6E01C10BF04DEC0BF0180E0C6E02C13A
:1018E0000BF04DEC0BF0190E0C6E03C10BF04DEC30
:1018F0000BF000C18EF101C18FF102C190F103C163
:1019000091F100C192F101C193F102C194F103C1BF
:1019100095F11A0E64EC0BF0E8CF00F11B0E64ECAD
:101920000BF0E8CF01F11C0E64EC0BF0E8CF02F1F4
:101930001D0E64EC0BF0E8CF03F1010103AFCFEF14
:101940000CF0E0EC31F01A0E0C6E00C10BF04DEC17
:101950000BF01B0E0C6E01C10BF04DEC0BF01C0ECE
:101960000C6E02C10BF04DEC0BF01D0E0C6E03C1A2
:101970000BF04DEC0BF01A0E64EC0BF0E8CF00F11D
:101980001B0E64EC0BF0E8CF01F11C0E64EC0BF0C5
:10199000E8CF02F11D0E64EC0BF0E8CF03F100C1BB
:1019A00096F101C197F102C198F103C199F1240E9A
:1019B000AC6E900EAB6E240EAC6E080EB86E000EC0
:1019C000B06E1F0EAF6E0401806B816B0F01900E25
:1019D000AB6E0F019D8A0301806B816BC26B8B9292
:1019E0004FEC37F04FEC37F031EC39F02DEC35F0AF
:1019F000200E64EC0BF0E8CF2FF505012F51FF0A04
:101A0000D8A40AEF0DF02F6B200E0C6E2FC50BF033
:101A10004DEC0BF00501010E306F3C0E316F250EC1
:101A200064EC0BF0E8CF00F1260E64EC0BF0E8CF8D
:101A300001F1270E64EC0BF0E8CF02F1280E64EC04
:101A40000BF0E8CF03F1010103AF41EF0DF0E0EC43
:101A500031F0250E0C6E00C10BF04DEC0BF0260E94
:101A60000C6E01C10BF04DEC0BF0270E0C6E02C199
:101A70000BF04DEC0BF0280E0C6E03C10BF04DEC8F
:101A80000BF000C157F501C158F502C159F503C16A
:101A90005AF500C15BF501C15CF502C15DF503C1FA
:101AA0005EF5290E64EC0BF0E8CF5FF5050160519F
:101AB0005F5DD8A05FC560F5210E64EC0BF0E8CF48
:101AC00000F1220E64EC0BF0E8CF01F1230E64EC80
:101AD0000BF0E8CF02F1240E64EC0BF0E8CF03F139
:101AE000010103AFA2EF0DF0E0EC31F0210E0C6E1E
:101AF00000C10BF04DEC0BF0220E0C6E01C10BF08F
:101B00004DEC0BF0230E0C6E02C10BF04DEC0BF004
:101B1000240E0C6E03C10BF04DEC0BF0210E64ECA7
:101B20000BF0E8CF00F1220E64EC0BF0E8CF01F1EE
:101B3000230E64EC0BF0E8CF02F1240E64EC0BF002
:101B4000E8CF03F100C161F501C162F502C163F59F
:101B500003C164F53EEC34F05BEC33F091EC32F011
:101B60001590C70E64EC0BF0E8CF00F1010100B155
:101B7000BDEF0DF01592BEEF0DF0158281AACCEFEE
:101B80000DF015B4C7EF0DF01580CCEF0DF070EC33
:101B900039F015A0D9EF39F007900001F28EF28CE0
:101BA00012AE03D012BC7AEF19F007B0F2EF2DF0AD
:101BB0000FB0B6EF26F010BEB6EF26F012B8B6EFB3
:101BC00026F000011650010AD8B4BEEF1DF081BA0C
:101BD000F2EF0DF000011650040AD8B437EF1CF0F4
:101BE000F8EF0DF000011650040AD8B4FAEF1DF01A
:101BF0000301805181197F0BD8B4F2EF2DF013EE61
:101C000000F081517F0BE126812BE7CFE8FFE00B4D
:101C1000D8B4F2EF2DF023EE82F0C2513F0BD9265B
:101C2000E7CFDFFFC22BDF50780AD8A4F2EF2DF008
:101C3000078092C100F193C101F194C102F195C1F5
:101C400003F10101040E046F000E056F000E066F14
:101C5000000E076FCBEC30F000AF38EF0EF0010153
:101C6000030E926F000E936F000E946F000E956F2F
:101C700003018251720AD8B437EF26F08251520A1A
:101C8000D8B437EF26F08251750AD8B437EF26F072
:101C90008251680AD8B4B6EF0EF08251630AD8B404
:101CA000ACEF2AF08251690AD8B404EF21F08251D6
:101CB0007A0AD8B417EF22F08251490AD8B4A3EFB8
:101CC00020F08251500AD8B4C1EF1FF08251700A3F
:101CD000D8B404EF20F08251540AD8B42FEF20F08A
:101CE0008251740AD8B475EF20F08251410AD8B4F9
:101CF000BBEF0FF082514B0AD8B4B8EF0EF082510F
:101D00006D0AD8B42BEF14F082514D0AD8B444EFC9
:101D100014F08251730AD8B467EF25F08251530A48
:101D2000D8B4CCEF25F082514C0AD8B4D3EF14F0DC
:101D30008251590AD8B47CEF13F012AE01D0128C44
:101D4000E3EF2AF0040114EE00F080517F0BE1264E
:101D500082C4E7FF802B120004010D0E826FA2ECFB
:101D60000EF00A0E826FA2EC0EF01200E1EF2AF0E4
:101D700004014B0E826FA2EC0EF004012C0E826F58
:101D8000A2EC0EF081B802D037B630D003018351F7
:101D9000430AD8B4FDEF0EF003018351630AD8B4AF
:101DA000FFEF0EF003018351520AD8B401EF0FF098
:101DB00003018351720AD8B403EF0FF0030183517A
:101DC000470AD8B405EF0FF003018351670AD8B46E
:101DD00007EF0FF003018351540AD8B409EF0FF055
:101DE00003018351740AD8B479EF0FF003018351D2
:101DF000550AD8B40BEF0FF083D037807BD03790E3
:101E000079D0378277D0379275D0378473D03794B2
:101E100071D037866FD084C330F185C331F186C36A
:101E200032F187C333F10101296B2EEC32F0A5ECBE
:101E300031F000C104F101C105F102C106F103C195
:101E400007F121EC32F0200EF86EF76AF66A09000D
:101E5000F5CF2CF10900F5CF2DF10900F5CF2EF1CA
:101E60000900F5CF2FF10900F5CF30F10900F5CFCA
:101E700031F10900F5CF32F10900F5CF33F101015D
:101E8000296B2EEC32F0A5EC31F0CBEC30F00101F7
:101E9000006752EF0FF0016752EF0FF0026752EF49
:101EA0000FF0036701D025D004014E0E826FA2EC23
:101EB0000EF004016F0E826FA2EC0EF004014D0EC5
:101EC000826FA2EC0EF00401610E826FA2EC0EF0A4
:101ED0000401740E826FA2EC0EF00401630E826F97
:101EE000A2EC0EF00401680E826FA2EC0EF0E1EF9E
:101EF0002AF03796CD0E0C6E37C00BF04DEC0BF080
:101F0000CD0E64EC0BF0E8CF37F037B006D004010B
:101F1000630E826FA2EC0EF005D00401430E826FB7
:101F2000A2EC0EF037B206D00401720E826FA2EC62
:101F30000EF005D00401520E826FA2EC0EF037B401
:101F400006D00401670E826FA2EC0EF005D00401EA
:101F5000470E826FA2EC0EF037B606D00401740E65
:101F6000826FA2EC0EF005D00401540E826FA2EC39
:101F70000EF0E1EF2AF00401410E826FA2EC0EF0A8
:101F800003018351310AD8B49CEF12F0030183514D
:101F9000320AD8B4CCEF11F003018351330AD8B41C
:101FA00055EF11F003018351340AD8B445EF10F016
:101FB00003018351350AD8B4E5EF0FF004013F0E59
:101FC000826FA2EC0EF0E1EF2AF003018451300A97
:101FD000D8B40BEF10F003018451310AD8B40EEFDE
:101FE00010F003018451650AD8B4FFEF0FF003012C
:101FF0008451640AD8B402EF10F00FEF10F038905B
:1020000003EF10F03880FB0E0C6E38C00BF04DEC77
:102010000BF00FEF10F08B900FEF10F08B8004019E
:10202000350E826FA2EC0EF004012C0E826FA2EC32
:102030000EF08BB023EF10F00401300E826FA2EC93
:102040000EF028EF10F00401310E826FA2EC0EF0BA
:1020500004012C0E826FA2EC0EF0FB0E64EC0BF070
:10206000E8CF38F038A03CEF10F00401640E826F26
:10207000A2EC0EF041EF10F00401650E826FA2ECAD
:102080000EF043EF10F0E1EF2AF0CC0E64EC0BF011
:10209000E8CF0BF004012C0E826FA2EC0EF00301CE
:1020A0008451310AD8B469EF10F003018451300A29
:1020B000D8B46BEF10F0030184514D0AD8B475EF1A
:1020C00010F003018451540AD8B47CEF10F093EF60
:1020D00010F08A8401D08A940BAE04D00BAC02D0ED
:1020E0000BBA21D0E00E0B1218D01F0E0B1685393B
:1020F000E844E00B0B1211D0E00E0B1621EC32F08D
:1021000085C332F186C333F10101296B2EEC32F025
:10211000A5EC31F000511F0B0B12CC0E0C6E0BC056
:102120000BF04DEC0BF00401340E826FA2EC0EF0BC
:1021300004012C0E826FA2EC0EF0CC0E64EC0BF0BE
:10214000E8CF1DF08AB406D00401300E826FA2ECF5
:102150000EF005D00401310E826FA2EC0EF00401E6
:102160002C0E826FA2EC0EF01D38E840070BE8CF72
:1021700082F40401300E8227A2EC0EF004012C0E32
:10218000826FA2EC0EF0E0EC31F01D501F0BE8CF97
:1021900000F169EC31F032C182F40401300E822783
:1021A000A2EC0EF033C182F40401300E8227A2ECBF
:1021B0000EF004012C0E826FA2EC0EF0E0EC31F078
:1021C00031C000F100AF0BD0FF0E016FFF0E026FA8
:1021D000FF0E036F04012D0E826FA2EC0EF069EC6E
:1021E00031F031C182F40401300E8227A2EC0EF0EE
:1021F00032C182F40401300E8227A2EC0EF033C10A
:1022000082F40401300E8227A2EC0EF004012C0EA1
:10221000826FA2EC0EF0E0EC31F030C000F169EC1E
:1022200031F031C182F40401300E8227A2EC0EF0AD
:1022300032C182F40401300E8227A2EC0EF033C1C9
:1022400082F40401300E8227A2EC0EF004012C0E61
:10225000826FA2EC0EF0E0EC31F032C000F100AF82
:102260000BD0FF0E016FFF0E026FFF0E036F040114
:102270002D0E826FA2EC0EF069EC31F031C182F4C8
:102280000401300E8227A2EC0EF032C182F4040168
:10229000300E8227A2EC0EF033C182F40401300E1E
:1022A0008227A2EC0EF0E1EF2AF0CB0E64EC0BF0EB
:1022B000E8CF0BF004012C0E826FA2EC0EF00301AC
:1022C0008451450AD8B479EF11F003018451440ACE
:1022D000D8B47CEF11F003018451300AD8B47FEFF9
:1022E00011F003018451310AD8B483EF11F08EEF5D
:1022F00011F00B9E88EF11F00B8E88EF11F0FC0EA1
:102300000B1688EF11F0FC0E0B160B8088EF11F006
:10231000CB0E0C6E0BC00BF04DEC0BF00401330E2A
:10232000826FA2EC0EF004012C0E826FA2EC0EF074
:10233000CB0E64EC0BF0E8CF1CF01CBEA7EF11F045
:102340000401450E826FA2EC0EF0ACEF11F0040117
:10235000440E826FA2EC0EF004012C0E826FA2ECF0
:102360000EF00401300E826FA2EC0EF004012C0E70
:10237000826FA2EC0EF01CB0C5EF11F00401300E1C
:10238000826FA2EC0EF0CAEF11F00401310E826FE1
:10239000A2EC0EF0E1EF2AF0CA0E64EC0BF0E8CFED
:1023A0000BF004012C0E826FA2EC0EF0030184519D
:1023B000450AD8B408EF12F003018451440AD8B496
:1023C0000BEF12F0030184514D0AD8B414EF12F050
:1023D00003018451410AD8B40EEF12F00301845175
:1023E000460AD8B411EF12F003018451560AD8B44A
:1023F0001CEF12F003018451500AD8B427EF12F0F9
:1024000003018451520AD8B42AEF12F033EF12F0CC
:102410000B9E2DEF12F00B8E2DEF12F00B9C2DEF7B
:1024200012F00B8C2DEF12F0FC0E0B1685C3E8FF9B
:10243000030B0B122DEF12F0C70E0B1685C3E8FF2E
:10244000070BE846E846E8460B122DEF12F00B8426
:102450002DEF12F00B942DEF12F0CA0E0C6E0BC084
:102460000BF04DEC0BF0CA0E64EC0BF0E8CF1BF058
:102470000401320E826FA2EC0EF004012C0E826F6A
:10248000A2EC0EF01BBE4CEF12F00401450E826F61
:10249000A2EC0EF051EF12F00401440E826FA2EC98
:1024A0000EF004012C0E826FA2EC0EF01BC0E8FFB0
:1024B000030BE8CF82F40401300E8227A2EC0EF069
:1024C00004012C0E826FA2EC0EF01BBC6FEF12F019
:1024D0000401410E826FA2EC0EF074EF12F00401C1
:1024E000460E826FA2EC0EF004012C0E826FA2EC5D
:1024F0000EF01BC0E8FF380BE842E842E842E8CFA4
:1025000082F40401300E8227A2EC0EF004012C0E9E
:10251000826FA2EC0EF01BB495EF12F00401520E84
:10252000826FA2EC0EF09AEF12F00401500E826F4F
:10253000A2EC0EF0E1EF2AF0C90E64EC0BF0E8CF4C
:102540000BF004012C0E826FA2EC0EF003018451FB
:10255000450AD8B4BAEF12F003018451440AD8B442
:10256000BDEF12F0030184514D0AD8B4C0EF12F050
:10257000CEEF12F00B9EC8EF12F00B8EC8EF12F0E8
:10258000F80E0B1685C3E8FF070B0B12C8EF12F00D
:10259000C90E0C6E0BC00BF04DEC0BF00401310EAC
:1025A000826FA2EC0EF004012C0E826FA2EC0EF0F2
:1025B000C90E64EC0BF0E8CF1AF01ABE06D0040185
:1025C000450E826FA2EC0EF005D00401440E826F1E
:1025D000A2EC0EF004012C0E826FA2EC0EF01AC0D9
:1025E000E8FF070BE8CF82F40401300E8227A2EC4B
:1025F0000EF004012C0E826FA2EC0EF00780E0ECCE
:1026000031F02CC0E8FF003B00430043030B69ECB2
:1026100031F033C182F40401300E8227A2EC0EF0B7
:1026200004012C0E826FA2EC0EF0E0EC31F02CC015
:1026300001F1019F019D2DC000F1010169EC31F014
:102640002FC182F40401300E8227A2EC0EF030C1BB
:1026500082F40401300E8227A2EC0EF031C182F424
:102660000401300E8227A2EC0EF032C182F4040184
:10267000300E8227A2EC0EF033C182F40401300E3A
:102680008227A2EC0EF004012C0E826FA2EC0EF059
:10269000E0EC31F02EC001F12FC000F1D8900133F1
:1026A0000033D89001330033010169EC31F02FC1C0
:1026B00082F40401300E8227A2EC0EF030C182F4C5
:1026C0000401300E8227A2EC0EF031C182F4040125
:1026D000300E8227A2EC0EF032C182F40401300EDB
:1026E0008227A2EC0EF033C182F40401300E82275F
:1026F000A2EC0EF0E1EF2AF0FC0E64EC0BF0E8CF58
:102700000BF003018351520AD8B4B3EF13F0030165
:102710008351720AD8B4B6EF13F003018351500A03
:10272000D8B4B9EF13F003018351700AD8B4BCEFE9
:1027300013F003018351550AD8B4BFEF13F003011E
:102740008351750AD8B4C2EF13F003018351430AD1
:10275000D8B4CBEF13F003018351630AD8B4CEEFA2
:1027600013F0D7EF13F00B90D1EF13F00B80D1EFF4
:1027700013F00B92D1EF13F00B82D1EF13F00B9407
:10278000D1EF13F00B84D1EF13F00B96D1EF13F0D0
:102790000B86D1EF13F00B98D1EF13F00B88D1EF2C
:1027A00013F0FC0E0C6E0BC00BF04DEC0BF00401A3
:1027B000590E826FA2EC0EF01190119211941198A3
:1027C000FC0E64EC0BF0E8CF0BF00BA011800BA219
:1027D00011820BA411840BA8118811A0F7EF13F03C
:1027E0000401520E826FA2EC0EF0FCEF13F0040114
:1027F000720E826FA2EC0EF011A806EF14F0040125
:10280000430E826FA2EC0EF00BEF14F00401630E86
:10281000826FA2EC0EF011A215EF14F00401500E1D
:10282000826FA2EC0EF01AEF14F00401700E826FAA
:10283000A2EC0EF011A424EF14F00401550E826FE7
:10284000A2EC0EF029EF14F00401750E826FA2ECD9
:102850000EF0E1EF2AF004016D0E826FA2EC0EF093
:1028600003018351300AD8B483EF14F0030183517C
:10287000310AD8B496EF14F003018351320AD8B468
:10288000A9EF14F0E3EF2AF004014D0E826FA2ECE1
:102890000EF021EC32F084C331F185C332F186C3EE
:1028A00033F10101296B2EEC32F0A5EC31F003017C
:1028B0008351300AD8B46BEF14F003018351310A0D
:1028C000D8B473EF14F003018351320AD8B47BEF0C
:1028D00014F0E3EF2AF0FD0E0C6E00C10BF04DEC8E
:1028E0000BF083EF14F0FE0E0C6E00C10BF04DECFC
:1028F0000BF096EF14F0FF0E0C6E00C10BF04DECD8
:102900000BF0A9EF14F00401300E826FA2EC0EF070
:1029100004012C0E826FA2EC0EF0E0EC31F0FD0E03
:1029200064EC0BF0E8CF00F1BAEF14F00401310EC3
:10293000826FA2EC0EF004012C0E826FA2EC0EF05E
:10294000E0EC31F0FE0E64EC0BF0E8CF00F1BAEFF2
:1029500014F00401320E826FA2EC0EF0E0EC31F0C4
:1029600004012C0E826FA2EC0EF0FF0E64EC0BF053
:10297000E8CF00F169EC31F031C182F40401300E8E
:102980008227A2EC0EF032C182F40401300E8227BD
:10299000A2EC0EF033C182F40401300E8227A2ECC7
:1029A0000EF0E1EF2AF003018351300AD8B427EF8B
:1029B0001AF003018351310AD8B465EF1BF003010B
:1029C0008351320AD8B4D3EF1BF003018351330A89
:1029D000D8B4E3EF1BF003018351340AD8B43EEFBF
:1029E0001CF003018351350AD8B412EF1EF0030125
:1029F0008351360AD8B440EF1EF003018351370AE1
:102A0000D8B4FFEF17F003018351380AD8B49DEF13
:102A100018F003018351440AD8B42BEF16F00301D8
:102A20008351640AD8B44BEF16F003018351460A70
:102A3000D8B417EF1DF0030183514D0AD8B478EFD5
:102A400016F0030183516D0AD8B492EF16F003011A
:102A500083515A0AD8B4DFEF1AF003018351490AAF
:102A6000D8B440EF1FF003018351500AD8B472EF7D
:102A70001EF003018351540AD8B4EBEF1EF003019A
:102A80008351630AD8B4B2EF16F003018351430AAD
:102A9000D8B4AAEF17F003018351730AD8B4B0EF8A
:102AA00016F003018351610AD8B478EF15F00301E1
:102AB0008351650AD8B477EF1AF003018351450AB0
:102AC000D8B485EF1AF003018351620AD8B493EFAA
:102AD0001AF003018351420AD8B4A1EF1AF003019E
:102AE0008351760AD8B4AFEF1AF0D8A4E3EF2AF0F6
:102AF00004014C0E826FA2EC0EF00401610E826F95
:102B0000A2EC0EF05BEC33F004012C0E826FA2EC11
:102B10000EF0E0EC31F0AFC500F1010169EC31F0ED
:102B200031C182F40401300E8227A2EC0EF032C1D2
:102B300082F40401300E8227A2EC0EF033C182F43D
:102B40000401300E8227A2EC0EF004012C0E826FDD
:102B5000A2EC0EF0E0EC31F0B0C500F1010169EC3F
:102B600031F031C182F40401300E8227A2EC0EF064
:102B700032C182F40401300E8227A2EC0EF033C180
:102B800082F40401300E8227A2EC0EF004012C0E18
:102B9000826FA2EC0EF0E0EC31F0B1C500F1010162
:102BA00069EC31F031C182F40401300E8227A2ECCD
:102BB0000EF032C182F40401300E8227A2EC0EF036
:102BC00033C182F40401300E8227A2EC0EF004011E
:102BD0002C0E826FA2EC0EF0E0EC31F0B2C500F1E9
:102BE000010169EC31F031C182F40401300E822719
:102BF000A2EC0EF032C182F40401300E8227A2EC66
:102C00000EF033C182F40401300E8227A2EC0EF0E4
:102C100004012C0E826FA2EC0EF0E0EC31F0B6C590
:102C200000F1010169EC31F031C182F40401300E90
:102C30008227A2EC0EF032C182F40401300E82270A
:102C4000A2EC0EF033C182F40401300E8227A2EC14
:102C50000EF06EEF1EF003018451300AD8B437EF46
:102C600016F003018451310AD8B43BEF16F01592E7
:102C700015963CEF16F01582C70E64EC0BF0E8CF0A
:102C800000F10101008115A20091C70E0C6E00C178
:102C90000BF04DEC0BF0C70E64EC0BF0E8CF00F13D
:102CA000010100B157EF16F0159258EF16F015829A
:102CB00004014C0E826FA2EC0EF00401640E826FD0
:102CC000A2EC0EF004012C0E826FA2EC0EF015B2F5
:102CD00071EF16F00401300E826FA2EC0EF076EF69
:102CE00016F00401310E826FA2EC0EF0E1EF2AF033
:102CF00021EC32F084C333F12EEC32F0A5EC31F04C
:102D0000200E0C6E00C10BF04DEC0BF000C12FF546
:102D100005012F51000A06E005012F51010A02E0CA
:102D2000BEEC33F004014C0E826FA2EC0EF00401F5
:102D30004D0E826FA2EC0EF004012C0E826FA2ECFD
:102D40000EF0E0EC31F02FC500F169EC31F033C149
:102D500082F40401300E8227A2EC0EF06EEF1EF01A
:102D6000D9EF39F004014C0E826FA2EC0EF0040191
:102D7000630E826FA2EC0EF091EC32F004012C0E87
:102D8000826FA2EC0EF0C7EC16F06EEF1EF0E0ECD6
:102D900031F0B5C500F10101003B0F0E001769ECE1
:102DA00031F033C182F40401300E8227A2EC0EF020
:102DB000B5C500F101010F0E0101001769EC31F0FA
:102DC00033C182F40401300E8227A2EC0EF004011C
:102DD0002D0E826FA2EC0EF0B4C500F10101003B94
:102DE0000F0E001769EC31F033C182F40401300E8C
:102DF0008227A2EC0EF0B4C500F101010F0E010113
:102E0000001769EC31F033C182F40401300E8227DF
:102E1000A2EC0EF004012D0E826FA2EC0EF0B3C5F1
:102E200000F10101003B0F0E001769EC31F033C1D6
:102E300082F40401300E8227A2EC0EF0B3C500F13B
:102E400001010F0E0101001769EC31F033C182F46A
:102E50000401300E8227A2EC0EF00401200E826FD6
:102E6000A2EC0EF0B2C500F10F0E0101001769ECE3
:102E700031F033C182F40401300E8227A2EC0EF04F
:102E80000401200E826FA2EC0EF0B1C500F1010129
:102E90000101003B0F0E001769EC31F033C182F4E1
:102EA0000401300E8227A2EC0EF0B1C500F1010141
:102EB0000F0E0101001769EC31F033C182F40401F7
:102EC000300E8227A2EC0EF004013A0E826FA2ECC3
:102ED0000EF0B0C500F10101003B0F0E001769ECC8
:102EE00031F033C182F40401300E8227A2EC0EF0DF
:102EF000B0C500F101010F0E0101001769EC31F0BE
:102F000033C182F40401300E8227A2EC0EF00401DA
:102F10003A0E826FA2EC0EF0AFC500F10101003B4A
:102F20000F0E001769EC31F033C182F40401300E4A
:102F30008227A2EC0EF0AFC500F101010F0E0017C1
:102F400069EC31F033C182F40401300E8227A2EC27
:102F50000EF0120084C3E8FF0F0BE83AE8CFB5F596
:102F600085C3E8FF0F0B0501B51387C3E8FF0F0BFF
:102F7000E83AE8CFB4F588C3E8FF0F0B0501B413B6
:102F80008AC3E8FF0F0BE83AE8CFB3F58BC3E8FF3D
:102F90000F0B0501B3138DC3E8FF0F0BE8CFB2F59C
:102FA0008FC3E8FF0F0BE83AE8CFB1F590C3E8FF15
:102FB0000F0B0501B11392C3E8FF0F0BE83AE8CFFE
:102FC000B0F593C3E8FF0F0B0501B01395C3E8FFFD
:102FD0000F0BE83AE8CFAFF596C3E8FF0F0B0501FA
:102FE000AF13FDEC32F004014C0E826FA2EC0EF038
:102FF0000401430E826FA2EC0EF0BCEF16F00784C2
:1030000004014C0E826FA2EC0EF00401370E826FA9
:10301000A2EC0EF004012C0E826FA2EC0EF0050162
:103020002E51130A06E005012E51170A0DE09AEF02
:1030300018F00101000E006F000E016F100E026FFC
:10304000000E036F2DEF18F00101000E006F000E4F
:10305000016F000E026F010E036F69EC31F02AC19F
:1030600082F40401300E8227A2EC0EF02BC182F410
:103070000401300E8227A2EC0EF02CC182F4040170
:10308000300E8227A2EC0EF02DC182F40401300E26
:103090008227A2EC0EF02EC182F40401300E8227AA
:1030A000A2EC0EF02FC182F40401300E8227A2ECB4
:1030B0000EF030C182F40401300E8227A2EC0EF033
:1030C00031C182F40401300E8227A2EC0EF032C12D
:1030D00082F40401300E8227A2EC0EF033C182F498
:1030E0000401300E8227A2EC0EF004012C0E826F38
:1030F000A2EC0EF00101100E006F000E016F000E29
:10310000026F000E036F69EC31F031C182F40401EB
:10311000300E8227A2EC0EF032C182F40401300E90
:103120008227A2EC0EF033C182F40401300E822714
:10313000A2EC0EF007946EEF1EF00501216B226BDE
:10314000236B246B04014C0E826FA2EC0EF0040181
:10315000380E826FA2EC0EF004012C0E826FA2ECEE
:103160000EF00101100E006F000E016F000E026FD5
:10317000000E036F69EC31F02AC182F40401300EB5
:103180008227A2EC0EF02BC182F40401300E8227BC
:10319000A2EC0EF02CC182F40401300E8227A2ECC6
:1031A0000EF02DC182F40401300E8227A2EC0EF045
:1031B0002EC182F40401300E8227A2EC0EF02FC142
:1031C00082F40401300E8227A2EC0EF030C182F4AA
:1031D0000401300E8227A2EC0EF031C182F404010A
:1031E000300E8227A2EC0EF032C182F40401300EC0
:1031F0008227A2EC0EF033C182F40401300E822744
:10320000A2EC0EF004012C0E826FA2EC0EF025C58C
:1032100000F126C501F127C502F128C503F101011E
:10322000100E046F000E056F000E066F000E076F84
:10323000FCEC30F000C133F501C134F502C135F5C5
:1032400003C136F569EC31F02AC182F40401300E75
:103250008227A2EC0EF02BC182F40401300E8227EB
:10326000A2EC0EF02CC182F40401300E8227A2ECF5
:103270000EF02DC182F40401300E8227A2EC0EF074
:103280002EC182F40401300E8227A2EC0EF02FC171
:1032900082F40401300E8227A2EC0EF030C182F4D9
:1032A0000401300E8227A2EC0EF031C182F4040139
:1032B000300E8227A2EC0EF032C182F40401300EEF
:1032C0008227A2EC0EF033C182F40401300E822773
:1032D000A2EC0EF0ACEC0EF00501336777EF19F0BD
:1032E000346777EF19F0356777EF19F0366702D05A
:1032F00016EF1AF0129E129C21C500F122C501F1B1
:1033000023C502F124C503F1899A400EC76E200E31
:10331000C66E9E96C69E0B0EC96EFF0E9EB602D05E
:10332000E82EFCD79E96C69E02C1C9FFFF0E9EB630
:1033300002D0E82EFCD79E96C69E01C1C9FFFF0EA3
:103340009EB602D0E82EFCD79E96C69E00C1C9FF4D
:10335000FF0E9EB602D0E82EFCD79E96C69EC9529E
:10336000FF0E9EB602D0E82EFCD70501100E326F7C
:10337000040114EE00F080517F0BE1269E96C69E5C
:10338000C952FF0E9EB602D0E82EFCD7C9CFE7FF88
:103390000401802B0501322FB8EF19F0898A33C55B
:1033A00000F134C501F135C502F136C503F1010163
:1033B000010E046F000E056F000E066F000E076F02
:1033C000CBEC30F000C133F501C134F502C135F565
:1033D00003C136F505013367F5EF19F03467F5EFF2
:1033E00019F03567F5EF19F0366702D016EF1AF0CD
:1033F00021C500F122C501F123C502F124C503F165
:103400000101100E046F000E056F000E066F000E16
:10341000076FD0EC30F000C121F501C122F502C1E7
:1034200023F503C124F5128EE3EF2AF00401450EC3
:10343000826FA2EC0EF004014F0E826FA2EC0EF030
:103440000401460E826FA2EC0EF06EEF1EF00784B0
:1034500031EC39F0E0EC31F02DC500F169EC31F0E0
:1034600004014C0E826FA2EC0EF00401300E826F4C
:10347000A2EC0EF004012C0E826FA2EC0EF031C112
:1034800082F40401300E8227A2EC0EF032C182F4E5
:103490000401300E8227A2EC0EF033C182F4040145
:1034A000300E8227A2EC0EF004012C0E826FA2ECEB
:1034B0000EF0E0EC31F02EC500F169EC31F031C1D5
:1034C00082F40401300E8227A2EC0EF032C182F4A5
:1034D0000401300E8227A2EC0EF033C182F4040105
:1034E000300E8227A2EC0EF007946EEF1EF004015E
:1034F0004C0E826FA2EC0EF00401650E826FA2ECFE
:103500000EF0D1EC34F06EEF1EF004014C0E826F21
:10351000A2EC0EF00401450E826FA2EC0EF0E8EC76
:1035200034F06EEF1EF004014C0E826FA2EC0EF030
:103530000401620E826FA2EC0EF016EC35F06EEF15
:103540001EF004014C0E826FA2EC0EF00401420E3C
:10355000826FA2EC0EF0FFEC34F06EEF1EF004016F
:103560004C0E826FA2EC0EF00401760E826FA2EC7C
:103570000EF004012C0E826FA2EC0EF0000125501B
:10358000FE0AD8B4D1EF1AF000012550FD0AD8B4D4
:10359000D8EF1AF00401300E826FA2EC0EF06EEF3D
:1035A0001EF00401310E826FA2EC0EF06EEF1EF0E1
:1035B0000401320E826FA2EC0EF06EEF1EF00401D9
:1035C0004C0E826FA2EC0EF004015A0E826FA2EC38
:1035D0000EF004012C0E826FA2EC0EF031EC39F0EB
:1035E000E0EC31F005012E51130A06E005012E51E1
:1035F000170A0DE010EF1BF00101000E006F000E26
:10360000016F100E026F000E036F10EF1BF001012F
:10361000000E006F000E016F000E026F010E036FAF
:103620000101100E046F000E056F000E066F000EF4
:10363000076FFCEC30F069EC31F02AC182F4040130
:10364000300E8227A2EC0EF02BC182F40401300E62
:103650008227A2EC0EF02CC182F40401300E8227E6
:10366000A2EC0EF02DC182F40401300E8227A2ECF0
:103670000EF02EC182F40401300E8227A2EC0EF06F
:103680002FC182F40401300E8227A2EC0EF030C16B
:1036900082F40401300E8227A2EC0EF031C182F4D4
:1036A0000401300E8227A2EC0EF032C182F4040134
:1036B000300E8227A2EC0EF033C182F40401300EEA
:1036C0008227A2EC0EF06EEF1EF0078404014C0E70
:1036D000826FA2EC0EF00401310E826FA2EC0EF0AC
:1036E00004012C0E826FA2EC0EF025C500F126C558
:1036F00001F127C502F128C503F10101100E046F85
:10370000000E056F000E066F000E076FFCEC30F028
:1037100069EC31F02AC182F40401300E8227A2EC58
:103720000EF02BC182F40401300E8227A2EC0EF0C1
:103730002CC182F40401300E8227A2EC0EF02DC1C0
:1037400082F40401300E8227A2EC0EF02EC182F426
:103750000401300E8227A2EC0EF02FC182F4040186
:10376000300E8227A2EC0EF030C182F40401300E3C
:103770008227A2EC0EF031C182F40401300E8227C0
:10378000A2EC0EF032C182F40401300E8227A2ECCA
:103790000EF033C182F40401300E8227A2EC0EF049
:1037A00007946EEF1EF0078404014C0E826FA2ECAA
:1037B0000EF00401320E826FA2EC0EF005EC37F031
:1037C00007946EEF1EF0078438B0E9EF1BF0FCEFB2
:1037D0001BF0010E166E04014C0E826FA2EC0EF06F
:1037E0000401330E826FA2EC0EF062EC37F0000E93
:1037F000166E079470EF1BF0020E166E62EC37F037
:103800008B800501010E306F3C0E316F01015E6B44
:103810005F6B606B616B626B636B646B656B666B3C
:10382000676B686B696B536B546BCF6ACE6A0F9A88
:103830000F9C0F9E030E166E04014C0E826FA2ECBD
:103840000EF00401330E826FA2EC0EF004012C0E78
:10385000826FA2EC0EF004012D0E826FA2EC0EF02E
:103860000401310E826FA2EC0EF0E1EF2AF062EC5F
:1038700037F0000E166E8B90E3EF2AF007840401F8
:103880004C0E826FA2EC0EF00401340E826FA2EC9B
:103890000EF004012C0E826FA2EC0EF021EC32F03F
:1038A00084C32AF185C32BF186C32CF187C32DF184
:1038B00088C32EF189C32FF18AC330F18BC331F154
:1038C0008CC332F18DC333F10101296B2EEC32F040
:1038D000A5EC31F0100E046F000E056F000E066FA0
:1038E000000E076FDCEC30F000C121F501C122F5BC
:1038F00002C123F503C124F5E4EC38F038C5AFF577
:1039000039C5B0F53AC5B1F53BC5B2F53CC5B3F51F
:103910003DC5B4F53EC5B5F5C7EC16F004012C0E57
:10392000826FA2EC0EF03FC500F140C501F141C528
:1039300002F142C503F10101000E046F000E056F94
:10394000010E066F000E076FFCEC30F069EC31F0F1
:103950002967ADEF1CF0B2EF1CF004012D0E826F51
:10396000A2EC0EF030C182F40401300E8227A2ECEA
:103970000EF031C182F40401300E8227A2EC0EF069
:1039800004012E0E826FA2EC0EF032C182F404010B
:10399000300E8227A2EC0EF033C182F40401300E07
:1039A0008227A2EC0EF004012C0E826FA2EC0EF026
:1039B000E0EC31F043C500F144C501F10DEC2CF011
:1039C00004012C0E826FA2EC0EF0E0EC31F045C544
:1039D00000F169EC31F031C182F40401300E82272C
:1039E000A2EC0EF032C182F40401300E8227A2EC68
:1039F0000EF033C182F40401300E8227A2EC0EF0E7
:103A000004012C0E826FA2EC0EF037C5E8FFE8B877
:103A100006D00401300E826FA2EC0EF005D0040136
:103A2000310E826FA2EC0EF007946EEF1EF021ECC7
:103A300032F085C32AF186C32BF187C32CF188C3EA
:103A40002DF189C32EF18AC32FF18BC330F18CC3C2
:103A500031F18DC332F18EC333F10101296B2EECAC
:103A600032F0A5EC31F00101010E046F000E056F7C
:103A7000000E066F000E076FCBEC30F0100E046FD7
:103A8000000E056F000E066F000E076FDCEC30F0C5
:103A900000C129F501C12AF502C12BF503C12CF59E
:103AA0008CEC36F004014C0E826FA2EC0EF0040197
:103AB000460E826FA2EC0EF004012C0E826FA2EC77
:103AC0000EF025C500F126C501F127C502F128C574
:103AD00003F10101100E046F000E056F000E066F5A
:103AE000000E076FFCEC30F069EC31F02AC182F473
:103AF0000401300E8227A2EC0EF02BC182F40401E7
:103B0000300E8227A2EC0EF02CC182F40401300E9C
:103B10008227A2EC0EF02DC182F40401300E822720
:103B2000A2EC0EF02EC182F40401300E8227A2EC2A
:103B30000EF02FC182F40401300E8227A2EC0EF0A9
:103B400030C182F40401300E8227A2EC0EF031C1A4
:103B500082F40401300E8227A2EC0EF032C182F40E
:103B60000401300E8227A2EC0EF033C182F404016E
:103B7000300E8227A2EC0EF06EEF1EF038B0C3EFCD
:103B80001DF0020E166E62EC37F000011650020AAC
:103B9000D8B4E1EF1DF005012F51010AD8B4D7EFD9
:103BA0001DF015B2DCEF1DF081BADCEF1DF0000E48
:103BB000166E1584E3EF2AF0050E166E1584D9EF04
:103BC00039F08B8001015E6B5F6B606B616B626BC8
:103BD000636B646B656B666B676B686B696B536B70
:103BE000546BCF6ACE6A0F9A0F9C0F9E030E166E0F
:103BF000E3EF2AF062EC37F005012F51010AD8B447
:103C000008EF1EF015B20DEF1EF081BA0DEF1EF099
:103C1000000E166E1584E3EF2AF0050E166E15845D
:103C2000D9EF39F004014C0E826FA2EC0EF00401C2
:103C3000350E826FA2EC0EF004012C0E826FA2EC06
:103C40000EF0E0EC31F00784B9C500F1079469EC9F
:103C500031F031C182F40401300E8227A2EC0EF063
:103C600032C182F40401300E8227A2EC0EF033C17F
:103C700082F40401300E8227A2EC0EF06EEF1EF0EB
:103C800025EC37F0E0EC31F037C500F169EC31F0AC
:103C900004014C0E826FA2EC0EF00401360E826F0E
:103CA000A2EC0EF004012C0E826FA2EC0EF031C1DA
:103CB00082F40401300E8227A2EC0EF032C182F4AD
:103CC0000401300E8227A2EC0EF033C182F404010D
:103CD000300E8227A2EC0EF06EEF1EF0ACEC0EF070
:103CE000E3EF2AF004014C0E826FA2EC0EF0040107
:103CF000500E826FA2EC0EF004012C0E826FA2EC2B
:103D00000EF085C32AF186C32BF187C32CF188C33B
:103D10002DF189C32EF18AC32FF18BC330F18CC3EF
:103D200031F18DC332F18EC333F101012EEC32F04B
:103D3000A5EC31F003018451530A0DE003018451D5
:103D40004D0A38E00401780E826FA2EC0EF0ACEC64
:103D50000EF0E3EF2AF00401530E826FA2EC0EF096
:103D6000250E0C6E00C10BF04DEC0BF0260E0C6E08
:103D700001C10BF04DEC0BF0270E0C6E02C10BF0E5
:103D80004DEC0BF0280E0C6E03C10BF04DEC0BF05C
:103D900000C157F501C158F502C159F503C15AF5E3
:103DA00000C15BF501C15CF502C15DF503C15EF5C3
:103DB0004FEF1FF004014D0E826FA2EC0EF0290EA2
:103DC0000C6E00C10BF04DEC0BF000C15FF500C1B3
:103DD00060F54FEF1FF004014C0E826FA2EC0EF065
:103DE0000401540E826FA2EC0EF004012C0E826FBF
:103DF000A2EC0EF084C32AF185C32BF186C32CF10B
:103E000087C32DF188C32EF189C32FF18AC330F106
:103E10008BC331F18DC332F18EC333F101012EEC2E
:103E200032F0A5EC31F00101000E046F000E056FB9
:103E3000010E066F000E076FDCEC30F0210E0C6EE9
:103E400000C10BF04DEC0BF0220E0C6E01C10BF01B
:103E50004DEC0BF0230E0C6E02C10BF04DEC0BF091
:103E6000240E0C6E03C10BF04DEC0BF000C161F59C
:103E700001C162F502C163F503C164F54FEF1FF0A4
:103E800004014C0E826FA2EC0EF00401490E826F09
:103E9000A2EC0EF004012C0E826FA2EC0EF0250EA7
:103EA00064EC0BF0E8CF00F1260E64EC0BF0E8CFE9
:103EB00001F1270E64EC0BF0E8CF02F1280E64EC60
:103EC0000BF0E8CF03F169EC31F02CEC2FF004019A
:103ED000730E826FA2EC0EF004012C0E826FA2EC26
:103EE0000EF0E0EC31F0290E64EC0BF0E8CF00F1BD
:103EF00069EC31F02CEC2FF004016D0E826FA2EC16
:103F00000EF004012C0E826FA2EC0EF05BC500F1E6
:103F10005CC501F15DC502F15EC503F169EC31F0EC
:103F20002CEC2FF00401730E826FA2EC0EF0040152
:103F30002C0E826FA2EC0EF0E0EC31F060C500F1C7
:103F400069EC31F02CEC2FF004016D0E826FA2ECC5
:103F50000EF004012C0E826FA2EC0EF061C500F190
:103F600062C501F163C502F164C503F1FEEC2AF0FC
:103F700004012C0E826FA2EC0EF0ACEC0EF0E3EF1D
:103F80002AF083C32AF184C32BF185C32CF186C3A5
:103F90002DF187C32EF188C32FF189C330F18AC375
:103FA00031F18BC332F18CC333F101012EEC32F0CD
:103FB000A5EC31F0160E0C6E00C10BF04DEC0BF0C1
:103FC000170E0C6E01C10BF04DEC0BF0180E0C6EC1
:103FD00002C10BF04DEC0BF0190E0C6E03C10BF08F
:103FE0004DEC0BF000C18EF101C18FF102C190F1D7
:103FF00003C191F100C192F101C193F102C194F1A9
:1040000003C195F1A3EF20F083C32AF184C32BF100
:1040100085C32CF186C32DF187C32EF188C32FF100
:1040200089C330F18AC331F18BC332F18CC333F1D0
:1040300001012EEC32F0A5EC31F000C18EF101C18E
:104040008FF102C190F103C191F100C192F101C160
:1040500093F102C194F103C195F1A3EF20F083C362
:104060002AF184C32BF185C32CF186C32DF187C3BC
:104070002EF188C32FF189C330F18AC331F18CC38B
:1040800032F18DC333F101012EEC32F0A5EC31F0A9
:104090000101000E046F000E056F010E066F000E89
:1040A000076FDCEC30F01A0E0C6E00C10BF04DEC1B
:1040B0000BF01B0E0C6E01C10BF04DEC0BF01C0E47
:1040C0000C6E02C10BF04DEC0BF01D0E0C6E03C11B
:1040D0000BF04DEC0BF000C196F101C197F102C15C
:1040E00098F103C199F1A3EF20F083C32AF184C3AF
:1040F0002BF185C32CF186C32DF187C32EF188C324
:104100002FF189C330F18AC331F18CC332F18DC3F1
:1041100033F101012EEC32F0A5EC31F00101000E7B
:10412000046F000E056F010E066F000E076FDCECCA
:1041300030F000C196F101C197F102C198F103C1BD
:1041400099F1A3EF20F0160E64EC0BF0E8CF00F12C
:10415000170E64EC0BF0E8CF01F1180E64EC0BF0D5
:10416000E8CF02F1190E64EC0BF0E8CF03F169EC33
:1041700031F02CEC2FF00401730E826FA2EC0EF0E4
:1041800004012C0E826FA2EC0EF08EC100F18FC1E3
:1041900001F190C102F191C103F169EC31F02CEC15
:1041A0002FF00401730E826FA2EC0EF004012C0EAE
:1041B000826FA2EC0EF01A0E64EC0BF0E8CF00F167
:1041C0001B0E64EC0BF0E8CF01F11C0E64EC0BF05D
:1041D000E8CF02F11D0E64EC0BF0E8CF03F1FEEC2A
:1041E0002AF004012C0E826FA2EC0EF096C100F1B1
:1041F00097C101F198C102F199C103F1FEEC2AF0D7
:10420000ACEC0EF0E3EF2AF00401690E826FA2EC31
:104210000EF004012C0E826FA2EC0EF00101040ED0
:10422000006F000E016F000E026F000E036F69EC4D
:1042300031F02CC182F40401300E8227A2EC0EF082
:104240002DC182F40401300E8227A2EC0EF02EC1A3
:1042500082F40401300E8227A2EC0EF02FC182F40A
:104260000401300E8227A2EC0EF030C182F404016A
:10427000300E8227A2EC0EF031C182F40401300E20
:104280008227A2EC0EF032C182F40401300E8227A4
:10429000A2EC0EF033C182F40401300E8227A2ECAE
:1042A0000EF004012C0E826FA2EC0EF00101060E3E
:1042B000006F000E016F000E026F000E036F69ECBD
:1042C00031F02CC182F40401300E8227A2EC0EF0F2
:1042D0002DC182F40401300E8227A2EC0EF02EC113
:1042E00082F40401300E8227A2EC0EF02FC182F47A
:1042F0000401300E8227A2EC0EF030C182F40401DA
:10430000300E8227A2EC0EF031C182F40401300E8F
:104310008227A2EC0EF032C182F40401300E822713
:10432000A2EC0EF033C182F40401300E8227A2EC1D
:104330000EF004012C0E826FA2EC0EF00101530E60
:10434000006F000E016F000E026F000E036F69EC2C
:1043500031F02CC182F40401300E8227A2EC0EF061
:104360002DC182F40401300E8227A2EC0EF02EC182
:1043700082F40401300E8227A2EC0EF02FC182F4E9
:104380000401300E8227A2EC0EF030C182F4040149
:10439000300E8227A2EC0EF031C182F40401300EFF
:1043A0008227A2EC0EF032C182F40401300E822783
:1043B000A2EC0EF033C182F40401300E8227A2EC8D
:1043C0000EF004012C0E826FA2EC0EF0200EF86E9F
:1043D000F76AF66A04010900F5CF82F4A2EC0EF048
:1043E0000900F5CF82F4A2EC0EF00900F5CF82F4BB
:1043F000A2EC0EF00900F5CF82F4A2EC0EF0090059
:10440000F5CF82F4A2EC0EF00900F5CF82F4A2EC15
:104410000EF00900F5CF82F4A2EC0EF00900F5CF02
:1044200082F4A2EC0EF0ACEC0EF0E3EF2AF0835134
:10443000630AD8A4E1EF2AF08451610AD8A4E1EF1D
:104440002AF085516C0AD8A4E1EF2AF08651410A7E
:104450003FE08651440A1BE08651420AD8B47BEF04
:1044600022F08651350AD8B46DEF2CF08651360A09
:10447000D8B4C2EF2CF08651370AD8B42BEF2DF008
:104480008651380AD8B489EF2DF0E1EF2AF0079869
:10449000079A04017A0E826FA2EC0EF00401780EE6
:1044A000826FA2EC0EF00401640E826FA2EC0EF09B
:1044B0000401550E826FA2EC0EF064EF22F00401AD
:1044C0004C0E826FA2EC0EF0ACEC0EF0E3EF2AF093
:1044D0000788079A04017A0E826FA2EC0EF004019D
:1044E000410E826FA2EC0EF00401610E826FA2EC0D
:1044F0000EF058EF22F00798078A04017A0E826FB7
:10450000A2EC0EF00401420E826FA2EC0EF0040148
:10451000610E826FA2EC0EF058EF22F00101666787
:1045200099EF22F0676799EF22F0686799EF22F020
:10453000696716D001014F67A5EF22F05067A5EF1C
:1045400022F05167A5EF22F052670AD00101000E58
:10455000006F000E016F000E026F000E036F12005D
:1045600011B80AD00101620E046F010E056F000E32
:10457000066F000E076F09D00101A70E046F020E2F
:10458000056F000E066F000E076F66C100F167C170
:1045900001F168C102F169C103F1CBEC30F003BF56
:1045A00042EF23F0119A119C0101000E046FA80E36
:1045B000056F550E066F020E076F66C100F167C1E9
:1045C00001F168C102F169C103F166C18AF167C1F5
:1045D0008BF168C18CF169C18DF1CBEC30F003BF78
:1045E0000BD00101000E8A6FA80E8B6F550E8C6FD9
:1045F000020E8D6F118A119C0E0E64EC0BF0E8CF49
:1046000018F10F0E64EC0BF0E8CF19F1100E64EC0A
:104610000BF0E8CF1AF1110E64EC0BF0E8CF1BF1B0
:1046200014EC30F08AC104F18BC105F18CC106F1A4
:104630008DC107F1CBEC30F00782D8EC2FF014ECF1
:1046400030F00792D8EC2FF08AC100F18BC101F154
:104650008CC102F18DC103F10792D8EC2FF0CC0E82
:10466000046FE00E056F870E066F050E076FCBEC2B
:1046700030F000C118F101C119F102C11AF103C1F2
:104680001BF140D013AA47EF23F0138E139A119C0D
:10469000119A0101800E006F1A0E016F060E026F53
:1046A000000E036F4FC104F150C105F151C106F175
:1046B00052C107F1CBEC30F003AF05D0E0EC31F0A4
:1046C000118C119A12000E0E64EC0BF0E8CF18F169
:1046D0000F0E64EC0BF0E8CF19F1100E64EC0BF048
:1046E000E8CF1AF1110E64EC0BF0E8CF1BF14FC1CB
:1046F00000F150C101F151C102F152C103F1078231
:10470000D8EC2FF018C100F119C101F11AC102F162
:104710001BC103F112000784BAC166F1BBC167F186
:10472000BCC168F1BDC169F14BC14FF14CC150F141
:104730004DC151F14EC152F157C159F158C15AF111
:10474000079401016667ACEF23F06767ACEF23F0D5
:104750006867ACEF23F0696716D001014F67B8EFC7
:1047600023F05067B8EF23F05167B8EF23F052679A
:104770000AD00101000E006F000E016F000E026FE3
:10478000000E036F120011B80AD00101620E046F0F
:10479000010E056F000E066F000E076F09D00101B4
:1047A000A70E046F020E056F000E066F000E076F56
:1047B00066C100F167C101F168C102F169C103F18D
:1047C000CBEC30F003BF44EF24F00101000E046F86
:1047D000A80E056F550E066F020E076F66C100F139
:1047E00067C101F168C102F169C103F166C18AF1D3
:1047F00067C18BF168C18CF169C18DF1CBEC30F0F0
:1048000003BF09D00101000E8A6FA80E8B6F550EF1
:104810008C6F020E8D6F14EC30F000C104F101C1F9
:1048200005F102C106F103C107F1000E006FA00EF1
:10483000016F980E026F7B0E036FFCEC30F000C12D
:1048400018F101C119F102C11AF103C11BF1000EE7
:10485000006FA00E016F980E026F7B0E036F8AC16E
:1048600004F18BC105F18CC106F18DC107F1FCEC9F
:1048700030F018C104F119C105F11AC106F11BC1CC
:1048800007F1CBEC30F012000101A80E006F610EB1
:10489000016F000E026F000E036F4FC104F150C193
:1048A00005F151C106F152C107F1CBEC30F003AF75
:1048B0000AD00101A80E006F610E016F000E026F99
:1048C000000E036F00D0C80E006FAF0E016F000E18
:1048D000026F000E036F4FC104F150C105F151C1C9
:1048E00006F152C107F1DCEC30F012000784BAC1C6
:1048F00066F1BBC167F1BCC168F1BDC169F14BC1D3
:104900004FF14CC150F14DC151F14EC152F157C15F
:1049100059F158C15AF107940101666797EF24F0E5
:10492000676797EF24F0686797EF24F0696716D000
:1049300001014F67A3EF24F05067A3EF24F0516704
:10494000A3EF24F052670AD00101000E006F000EA1
:10495000016F000E026F000E036F120011B80AD033
:104960000101620E046F010E056F000E066F000E4E
:10497000076F09D00101A70E046F020E056F000E2C
:10498000066F000E076F66C100F167C101F168C1D3
:1049900002F169C103F1CBEC30F003BF59EF25F010
:1049A0000101000E046FA80E056F550E066F020E72
:1049B000076F66C100F167C101F168C102F169C109
:1049C00003F166C18AF167C18BF168C18CF169C1DD
:1049D0008DF1CBEC30F003BF09D00101000E8A6FDE
:1049E000A80E8B6F550E8C6F020E8D6F010E006F2F
:1049F000000E016F000E026F000E036F8AC104F1FA
:104A00008BC105F18CC106F18DC107F1FCEC30F0D2
:104A100018C104F119C105F11AC106F11BC107F152
:104A200069EC31F02AC182F40401300E8227A2EC35
:104A30000EF02BC182F40401300E8227A2EC0EF09E
:104A40002CC182F40401300E8227A2EC0EF02DC19D
:104A500082F40401300E8227A2EC0EF02EC182F403
:104A60000401300E8227A2EC0EF02FC182F4040163
:104A7000300E8227A2EC0EF030C182F40401300E19
:104A80008227A2EC0EF031C182F40401300E82279D
:104A9000A2EC0EF032C182F40401300E8227A2ECA7
:104AA0000EF033C182F40401300E8227A2EC0EF026
:104AB00012004FC100F150C101F151C102F152C1C8
:104AC00003F1010169EC31F02CEC2FF0120004012C
:104AD000730E826FA2EC0EF004012C0E826FA2EC1A
:104AE0000EF0078462C166F163C167F164C168F1C9
:104AF00065C169F14BC14FF14CC150F14DC151F14C
:104B00004EC152F157C159F158C15AF107948DEC79
:104B100025F0ACEC0EF0E3EF2AF066C100F167C1BE
:104B200001F168C102F169C103F1010169EC31F0E1
:104B30002CEC2FF00401630E826FA2EC0EF0040146
:104B40002C0E826FA2EC0EF04FC100F150C101F1AA
:104B500051C102F152C103F1010169EC31F02CECB9
:104B60002FF00401660E826FA2EC0EF004012C0EF1
:104B7000826FA2EC0EF0E0EC31F059C100F15AC1A5
:104B800001F1010169EC31F02CEC2FF00401740EFD
:104B9000826FA2EC0EF0120010820401530E826F9D
:104BA000A2EC0EF004012C0E826FA2EC0EF083C377
:104BB0002AF184C32BF185C32CF186C32DF187C361
:104BC0002EF188C32FF189C330F18AC331F18BC331
:104BD00032F18CC333F101012EEC32F0A5EC31F04F
:104BE00000C166F101C167F102C168F103C169F159
:104BF0008EC32AF18FC32BF190C32CF191C32DF1F9
:104C000092C32EF193C32FF194C330F195C331F1C8
:104C100096C332F197C333F101012EEC32F0A5ECCB
:104C200031F000C14FF101C150F102C151F103C196
:104C300052F121EC32F099C32FF19AC330F19BC3AA
:104C400031F19CC332F19DC333F101012EEC32F0FE
:104C5000A5EC31F000C159F101C15AF18DEC25F0FC
:104C600004012C0E826FA2EC0EF047EF26F0118E9D
:104C70001CA002D01CAE108C1BBE02D01BA4108E38
:104C800003018251520A02E10F8201D00F92825138
:104C9000750A02E1108401D010948251550A02E194
:104CA000108601D010968351310A03E113821384D8
:104CB00002D01392139403018351660A01E056D087
:104CC0000401660E826FA2EC0EF004012C0E826FBE
:104CD000A2EC0EF08BEC23F069EC31F02AC182F4E7
:104CE0000401300E8227A2EC0EF02BC182F40401E5
:104CF000300E8227A2EC0EF02CC182F40401300E9B
:104D00008227A2EC0EF02DC182F40401300E82271E
:104D1000A2EC0EF02EC182F40401300E8227A2EC28
:104D20000EF02FC182F40401300E8227A2EC0EF0A7
:104D300030C182F40401300E8227A2EC0EF031C1A2
:104D400082F40401300E8227A2EC0EF032C182F40C
:104D50000401300E8227A2EC0EF033C182F404016C
:104D6000300E8227A2EC0EF0E1EF2AF011A003D062
:104D700011A401D01084078410B220EF27F010A4F2
:104D800004EF27F0BAC166F1BBC167F1BCC168F19D
:104D9000BDC169F1BEC16AF1BFC16BF1C0C16CF1A7
:104DA000C1C16DF1C2C16EF1C3C16FF1C4C170F177
:104DB000C5C171F1C6C172F1C7C173F1C8C174F147
:104DC000C9C175F1CAC176F1CBC177F1CCC178F117
:104DD000CDC179F1CEC17AF1CFC17BF1D0C17CF1E7
:104DE000D1C17DF1D2C17EF1D3C17FF1D4C180F1B7
:104DF000D5C181F1D6C182F1D7C183F1D8C184F187
:104E0000D9C185F10CEF27F062C166F163C167F18A
:104E100064C168F165C169F1BAC186F1BBC187F1AE
:104E2000BCC188F1BDC189F14BC14FF14CC150F1FA
:104E30004DC151F14EC152F157C159F158C15AF10A
:104E400007940FA042EF27F0010196672FEF27F09C
:104E500097672FEF27F098672FEF27F0996733EFC9
:104E600027F042EF27F08EEC22F096C104F197C1B3
:104E700005F198C106F199C107F1CBEC30F003BF01
:104E8000A7EF2AF08EEC22F00101000E046F000E55
:104E9000056F010E066F000E076FFCEC30F011A0DD
:104EA0002AD011A228D069EC31F0296701D005D0B1
:104EB00004012D0E826FA2EC0EF030C182F40401C9
:104EC000300E8227A2EC0EF031C182F40401300EC4
:104ED0008227A2EC0EF032C182F40401300E822748
:104EE000A2EC0EF033C182F40401300E8227A2EC52
:104EF0000EF0ACEC0EF012A8C5D012981DC01EF03A
:104F00001E3A1E42070E1E1600011E50000AD8B49B
:104F10000EEF28F000011E50010AD8B49AEF27F0D6
:104F200000011E50020AD8B498EF27F040EF28F095
:104F300040EF28F0E0EC31F02EC001F12FC000F17D
:104F4000D89001330033D890013300330101630E50
:104F5000046F000E056F000E066F000E076FFCEC6D
:104F600030F0280E046F000E056F000E066F000E65
:104F7000076FCBEC30F000C131F0E0EC31F02CC029
:104F800001F1019F019D2DC000F10101A40E046FEC
:104F9000000E056F000E066F000E076FFCEC30F080
:104FA00000C130F000C104F101C105F102C106F1F8
:104FB00003C107F1640E006F000E016F000E026F57
:104FC000000E036FCBEC30F0050E046F000E056F82
:104FD000000E066F000E076FFCEC30F000C104F10C
:104FE00001C105F102C106F103C107F1E0EC31F0A6
:104FF00031C000F1CBEC30F000C132F032C0E8FF3C
:10500000050F315C03E78A8440EF28F032C0E8FFE7
:105010000A0F315C01E68A9440EF28F000C124F1C8
:1050200001C125F102C126F103C127F1E0EC31F005
:10503000E6EC31F01D501F0BE8CF00F10101640ECA
:10504000046F000E056F000E066F000E076FDCEC9C
:1050500030F024C104F125C105F126C106F127C1B4
:1050600007F1CBEC30F003BF02D08A9401D08A84E0
:1050700024C100F125C101F126C102F127C103F1CC
:10508000E3EF2AF000C124F101C125F102C126F1AC
:1050900003C127F110AE4DD0109E00C108F101C12F
:1050A00009F102C10AF103C10BF169EC31F030C121
:1050B000E2F131C1E3F132C1E4F133C1E5F108C1FC
:1050C00000F109C101F10AC102F10BC103F10101B3
:1050D0006C0E046F070E056F000E066F000E076F53
:1050E000CBEC30F003BF04D00101550EE66F1CD0AD
:1050F00008C100F109C101F10AC102F10BC103F1BC
:105100000101A40E046F060E056F000E066F000E5F
:10511000076FCBEC30F003BF04D001017F0EE66FC8
:1051200003D00101FF0EE66F1F8E11AEA7EF2AF02C
:10513000119E24C100F125C101F126C102F127C150
:1051400003F111A005D011A203D00FB0A7EF2AF0F0
:1051500010A4B2EF28F00401750E826FA2EC0EF0DD
:10516000B7EF28F00401720E826FA2EC0EF004017A
:105170002C0E826FA2EC0EF069EC31F02967C6EFBD
:1051800028F00401200E826FC9EF28F004012D0ED3
:10519000826FA2EC0EF030C182F40401300E82273F
:1051A000A2EC0EF031C182F40401300E8227A2EC91
:1051B0000EF004012E0E826FA2EC0EF032C182F4CA
:1051C0000401300E8227A2EC0EF033C182F40401F8
:1051D000300E8227A2EC0EF004016D0E826FA2EC5D
:1051E0000EF004012C0E826FA2EC0EF04FC100F104
:1051F00050C101F151C102F152C103F1010169EC49
:1052000031F02CEC2FF00401480E826FA2EC0EF06E
:1052100004017A0E826FA2EC0EF004012C0E826F54
:10522000A2EC0EF066C100F167C101F168C102F1A4
:1052300069C103F1010169EC31F02CEC2FF004019C
:10524000630E826FA2EC0EF004012C0E826FA2ECB2
:105250000EF066C100F167C101F168C102F169C1D8
:1052600003F101010A0E046F000E056F000E066FB8
:10527000000E076FDCEC30F0000E046F120E056FAD
:10528000000E066F000E076FFCEC30F069EC31F099
:105290002AC182F40401300E8227A2EC0EF02BC149
:1052A00082F40401300E8227A2EC0EF02CC182F4AD
:1052B0000401300E8227A2EC0EF02DC182F404010D
:1052C000300E8227A2EC0EF02EC182F40401300EC3
:1052D0008227A2EC0EF02FC182F40401300E822747
:1052E000A2EC0EF030C182F40401300E8227A2EC51
:1052F0000EF004012E0E826FA2EC0EF031C182F48A
:105300000401300E8227A2EC0EF032C182F40401B7
:10531000300E8227A2EC0EF033C182F40401300E6D
:105320008227A2EC0EF00401730E826FA2EC0EF045
:1053300004012C0E826FA2EC0EF0E0EC31F059C1AA
:1053400000F15AC101F10DEC2CF003018351320A36
:1053500001E027D004012C0E826FA2EC0EF0E0ECED
:1053600031F00784B9C500F1079469EC31F031C11F
:1053700082F40401300E8227A2EC0EF032C182F4D6
:105380000401300E8227A2EC0EF033C182F4040136
:10539000300E8227A2EC0EF00401420E826FA2ECC6
:1053A0000EF013A223EF2AF004012C0E826FA2EC60
:1053B0000EF086C166F187C167F188C168F189C1C5
:1053C00069F18EEC22F00101000E046F000E056FF2
:1053D000010E066F000E076FFCEC30F069EC31F047
:1053E0002967F8EF29F00401200E826FFBEF29F006
:1053F00004012D0E826FA2EC0EF030C182F4040184
:10540000300E8227A2EC0EF031C182F40401300E7E
:105410008227A2EC0EF004012E0E826FA2EC0EF099
:1054200032C182F40401300E8227A2EC0EF033C1A7
:1054300082F40401300E8227A2EC0EF004016D0EFE
:10544000826FA2EC0EF003018351460A01E007D0FF
:1054500004012C0E826FA2EC0EF076EC24F013A463
:1054600056EF2AF004012C0E826FA2EC0EF013AC62
:1054700044EF2AF00401500E826FA2EC0EF0139C50
:105480001398139A56EF2AF013AE51EF2AF0040145
:10549000460E826FA2EC0EF0139E1398139A56EFED
:1054A0002AF00401530E826FA2EC0EF038B06DEFBB
:1054B0002AF004012C0E826FA2EC0EF08BB068EF84
:1054C0002AF00401440E826FA2EC0EF06DEF2AF078
:1054D0000401530E826FA2EC0EF00FB273EF2AF0AC
:1054E0000FA0A5EF2AF004012C0E826FA2EC0EF0A3
:1054F000200EF86EF76AF66A04010900F5CF82F40F
:10550000A2EC0EF00900F5CF82F4A2EC0EF0090037
:10551000F5CF82F4A2EC0EF00900F5CF82F4A2ECF4
:105520000EF00900F5CF82F4A2EC0EF00900F5CFE1
:1055300082F4A2EC0EF00900F5CF82F4A2EC0EF09A
:105540000900F5CF82F4A2EC0EF0ACEC0EF00F9057
:10555000109E1298E3EF2AF00401630E826FA2EC12
:105560000EF004012C0E826FA2EC0EF0E9EC2AF092
:1055700004012C0E826FA2EC0EF05CEC2BF0040107
:105580002C0E826FA2EC0EF0D8EC2BF004012C0E46
:10559000826FA2EC0EF00101F80E006FCD0E016FCC
:1055A000660E026F030E036FFEEC2AF004012C0E50
:1055B000826FA2EC0EF0EEEC2BF0ACEC0EF0E3EF11
:1055C0002AF0ACEC0EF00301C26B07901092F2EFE0
:1055D0002DF0D8900E0E64EC0BF0E8CF00F10F0E1A
:1055E00064EC0BF0E8CF01F1100E64EC0BF0E8CFA7
:1055F00002F1110E64EC0BF0E8CF03F10101000E93
:10560000046F000E056F010E066F000E076FFCECB5
:1056100030F069EC31F02AC182F40401300E8227A7
:10562000A2EC0EF02BC182F40401300E8227A2EC12
:105630000EF02CC182F40401300E8227A2EC0EF091
:105640002DC182F40401300E8227A2EC0EF02EC18F
:1056500082F40401300E8227A2EC0EF02FC182F4F6
:105660000401300E8227A2EC0EF030C182F4040156
:10567000300E8227A2EC0EF031C182F40401300E0C
:105680008227A2EC0EF004012E0E826FA2EC0EF027
:1056900032C182F40401300E8227A2EC0EF033C135
:1056A00082F40401300E8227A2EC0EF004016D0E8C
:1056B000826FA2EC0EF01200120E64EC0BF0E8CF39
:1056C00000F1130E64EC0BF0E8CF01F1140E64EC62
:1056D0000BF0E8CF02F1150E64EC0BF0E8CF03F10C
:1056E00001010A0E046F000E056F000E066F000E1A
:1056F000076FDCEC30F0000E046F120E056F000E29
:10570000066F000E076FFCEC30F069EC31F02AC137
:1057100082F40401300E8227A2EC0EF02BC182F439
:105720000401300E8227A2EC0EF02CC182F4040199
:10573000300E8227A2EC0EF02DC182F40401300E4F
:105740008227A2EC0EF02EC182F40401300E8227D3
:10575000A2EC0EF02FC182F40401300E8227A2ECDD
:105760000EF030C182F40401300E8227A2EC0EF05C
:1057700004012E0E826FA2EC0EF031C182F40401FE
:10578000300E8227A2EC0EF032C182F40401300EFA
:105790008227A2EC0EF033C182F40401300E82277E
:1057A000A2EC0EF00401730E826FA2EC0EF0120058
:1057B0000A0E64EC0BF0E8CF00F10B0E64EC0BF07A
:1057C000E8CF01F10C0E64EC0BF0E8CF02F10D0E06
:1057D00064EC0BF0E8CF03F10DEF2CF0060E64EC57
:1057E0000BF0E8CF00F1070E64EC0BF0E8CF01F10D
:1057F000080E64EC0BF0E8CF02F1090E64EC0BF03C
:10580000E8CF03F10DEF2CF00101E0EC31F007845B
:1058100057C100F158C101F107940101E80E046F6E
:10582000800E056F000E066F000E076FDCEC30F087
:10583000000E046F040E056F000E066F000E076F5A
:10584000FCEC30F0880E046F130E056F000E066F2F
:10585000000E076FCBEC30F00A0E046F000E056FE0
:10586000000E066F000E076FFCEC30F069EC31F0B3
:105870000101296741EF2CF00401200E826F44EFF3
:105880002CF004012D0E826FA2EC0EF030C182F4D8
:105890000401300E8227A2EC0EF031C182F4040123
:1058A000300E8227A2EC0EF032C182F40401300ED9
:1058B0008227A2EC0EF004012E0E826FA2EC0EF0F5
:1058C00033C182F40401300E8227A2EC0EF00401F1
:1058D000430E826FA2EC0EF0120087C32AF188C338
:1058E0002BF189C32CF18AC32DF18BC32EF18CC30C
:1058F0002FF18DC330F18EC331F190C332F191C3DA
:1059000033F10101296B2EEC32F0A5EC31F00101ED
:10591000000E046F000E056F010E066F000E076F7C
:10592000DCEC30F00E0E0C6E00C10BF04DEC0BF009
:105930000F0E0C6E01C10BF04DEC0BF0100E0C6E47
:1059400002C10BF04DEC0BF0110E0C6E03C10BF00D
:105950004DEC0BF004017A0E826FA2EC0EF0040104
:105960002C0E826FA2EC0EF00401350E826FA2ECB9
:105970000EF004012C0E826FA2EC0EF0E9EC2AF07E
:1059800064EF22F087C32AF188C32BF189C32CF17D
:105990008AC32DF18BC32EF18CC32FF18DC330F14F
:1059A0008EC331F190C332F191C333F10101296B00
:1059B0002EEC32F0A5EC31F0880E046F130E056F5B
:1059C000000E066F000E076FD0EC30F0000E046F73
:1059D000040E056F000E066F000E076FDCEC30F052
:1059E0000101E80E046F800E056F000E066F000EB9
:1059F000076FFCEC30F00A0E0C6E00C10BF04DECA2
:105A00000BF00B0E0C6E01C10BF04DEC0BF00C0EFD
:105A10000C6E02C10BF04DEC0BF00D0E0C6E03C1C1
:105A20000BF04DEC0BF004017A0E826FA2EC0EF03D
:105A300004012C0E826FA2EC0EF00401360E826F70
:105A4000A2EC0EF004012C0E826FA2EC0EF0D8EC4A
:105A50002BF064EF22F087C32AF188C32BF189C3AE
:105A60002CF18AC32DF18BC32EF18CC32FF18DC382
:105A700030F18FC331F190C332F191C333F10101A1
:105A80002EEC32F0A5EC31F0000E046F120E056F13
:105A9000000E066F000E076FDCEC30F001010A0EFD
:105AA000046F000E056F000E066F000E076FFCEC12
:105AB00030F0120E0C6E00C10BF04DEC0BF0130E1B
:105AC0000C6E01C10BF04DEC0BF0140E0C6E02C10C
:105AD0000BF04DEC0BF0150E0C6E03C10BF04DEC02
:105AE0000BF004017A0E826FA2EC0EF004012C0E72
:105AF000826FA2EC0EF00401370E826FA2EC0EF062
:105B000004012C0E826FA2EC0EF05CEC2BF064EF23
:105B100022F087C32AF188C32BF189C32CF18AC3F1
:105B20002DF18BC32EF18CC32FF18DC330F18EC3B9
:105B300031F190C332F191C333F10101296B2EECA5
:105B400032F0A5EC31F0880E046F130E056F000ED5
:105B5000066F000E076FD0EC30F0000E046F040EDD
:105B6000056F000E066F000E076FDCEC30F00101D0
:105B7000E80E046F800E056F000E066F000E076FB3
:105B8000FCEC30F0060E0C6E00C10BF04DEC0BF08F
:105B9000070E0C6E01C10BF04DEC0BF0080E0C6EF5
:105BA00002C10BF04DEC0BF0090E0C6E03C10BF0B3
:105BB0004DEC0BF004017A0E826FA2EC0EF00401A2
:105BC0002C0E826FA2EC0EF00401380E826FA2EC54
:105BD0000EF004012C0E826FA2EC0EF0EEEC2BF016
:105BE00064EF22F007A865EF2EF00101800E006F30
:105BF0001A0E016F060E026F000E036F4BC104F107
:105C00004CC105F14DC106F14EC107F1CBEC30F0AE
:105C100003BFABEF2EF026EC2FF04BC100F14CC1CF
:105C200001F14DC102F14EC103F10782D8EC2FF012
:105C300018C104F119C105F11AC106F11BC107F120
:105C4000F80E006FCD0E016F660E026F030E036F2C
:105C5000CBEC30F00E0E0C6E00C10BF04DEC0BF0E7
:105C60000F0E0C6E01C10BF04DEC0BF0100E0C6E14
:105C700002C10BF04DEC0BF0110E0C6E03C10BF0DA
:105C80004DEC0BF007840101E0EC31F057C100F15D
:105C900058C101F107940A0E0C6E00C10BF04DECD7
:105CA0000BF00B0E0C6E01C10BF04DEC0BF00C0E5B
:105CB0000C6E02C10BF04DEC0BF00D0E0C6E03C11F
:105CC0000BF04DEC0BF0ABEF2EF007AAABEF2EF084
:105CD00007840101E0EC31F057C100F158C101F136
:105CE0000794060E0C6E00C10BF04DEC0BF0070E86
:105CF0000C6E01C10BF04DEC0BF0080E0C6E02C1E6
:105D00000BF04DEC0BF0090E0C6E03C10BF04DECDB
:105D10000BF0078462C100F163C101F164C102F1BB
:105D200065C103F10794120E0C6E00C10BF04DEC2F
:105D30000BF0130E0C6E01C10BF04DEC0BF0140EBA
:105D40000C6E02C10BF04DEC0BF0150E0C6E03C186
:105D50000BF04DEC0BF00798079A04018051811964
:105D60007F0B0DE09EA8FED714EE00F081517F0B53
:105D7000E126E750812B0F01AD6EADEF2EF005014E
:105D80002F51000AD8B4EEEF2EF081BAD3EF2EF0E7
:105D900015B2EEEF2EF005012F51010AD8B4ECEF49
:105DA0002EF0E5EF2EF005012F51000AD8B4D9EFFF
:105DB00039F005012F51010AD8B4ECEF2EF00001A3
:105DC0001650050AD8B4D9EF39F081B8EEEF2EF0AD
:105DD0005BEC33F001EC34F070EC39F0D0EF0DF007
:105DE00018C100F119C101F11AC102F11BC103F17F
:105DF000000E046F000E056F010E066F000E076F98
:105E0000FCEC30F029A11BEF2FF02051D8B41BEF90
:105E10002FF018C100F119C101F11AC102F11BC123
:105E200003F1000E046F000E056F0A0E066F000EE0
:105E3000076FFCEC30F01200010104510013055112
:105E40000113065102130751031312000101186BCD
:105E5000196B1A6B1B6B12002AC182F40401300EFD
:105E60008227A2EC0EF02BC182F40401300E8227AF
:105E7000A2EC0EF02CC182F40401300E8227A2ECB9
:105E80000EF02DC182F40401300E8227A2EC0EF038
:105E90002EC182F40401300E8227A2EC0EF02FC135
:105EA00082F40401300E8227A2EC0EF030C182F49D
:105EB0000401300E8227A2EC0EF031C182F40401FD
:105EC000300E8227A2EC0EF032C182F40401300EB3
:105ED0008227A2EC0EF033C182F40401300E822737
:105EE000A2EC0EF012002FC182F40401300E8227C2
:105EF000A2EC0EF030C182F40401300E8227A2EC35
:105F00000EF031C182F40401300E8227A2EC0EF0B3
:105F100032C182F40401300E8227A2EC0EF033C1AC
:105F200082F40401300E8227A2EC0EF01200060E5D
:105F3000216E060E226E060E236E212E9DEF2FF08F
:105F4000222E9DEF2FF0232E9DEF2FF08B84020E3B
:105F5000216E020E226E020E236E212EADEF2FF067
:105F6000222EADEF2FF0232EADEF2FF08B941200E9
:105F7000FF0E226E22C023F0030E216E8B84212E91
:105F8000BEEF2FF0030E216E232EBEEF2FF08B9469
:105F900022C023F0030E216E212ECCEF2FF0030E32
:105FA000216E233ECCEF2FF0222EBAEF2FF01200FD
:105FB0000101005305E1015303E1025301E1002B0C
:105FC0009BEC30F0E0EC31F03951006F3A51016F49
:105FD000420E046F4B0E056F000E066F000E076F2A
:105FE000DCEC30F000C104F101C105F102C106F1A1
:105FF00003C107F118C100F119C101F11AC102F181
:106000001BC103F107B209EF30F0D0EC30F00BEF19
:1060100030F0CBEC30F000C118F101C119F102C130
:106020001AF103C11BF11200E0EC31F059C100F18B
:106030005AC101F1060E64EC0BF0E8CF04F1070E33
:1060400064EC0BF0E8CF05F1080E64EC0BF0E8CF40
:1060500006F1090E64EC0BF0E8CF07F1CBEC30F061
:1060600000C124F101C125F102C126F103C127F1CC
:10607000290E046F000E056F000E066F000E076FED
:10608000DCEC30F0EE0E046F430E056F000E066F71
:10609000000E076FD0EC30F024C104F125C105F1EA
:1060A00026C106F127C107F1DCEC30F000C11CF17C
:1060B00001C11DF102C11EF103C11FF1120E64ECFA
:1060C0000BF0E8CF04F1130E64EC0BF0E8CF05F110
:1060D000140E64EC0BF0E8CF06F1150E64EC0BF037
:1060E000E8CF07F10D0E006F000E016F000E026F7A
:1060F000000E036FDCEC30F0180E046F000E056F1D
:10610000000E066F000E076FFCEC30F01CC104F1AE
:106110001DC105F11EC106F11FC107F1D0EC30F021
:106120006A0E046F2A0E056F000E066F000E076FD1
:10613000CBEC30F01200BF0EFA6E200E3A6F396BC6
:10614000D8900037013702370337D8B0ACEF30F0C2
:106150003A2FA1EF30F039073A070353D8B41200B1
:106160000331070B80093F6F03390F0B010F396FA4
:1061700080EC5FF0406F390580EC5FF0405D405F80
:10618000396B3F33D8B0392739333FA9C1EF30F0ED
:10619000405139271200010105EC32F0D8B012004D
:1061A000010103510719346FC8EC31F0D890075141
:1061B000031934AF800F12000101346BECEC31F0A5
:1061C000D8A002EC32F0D8B01200D7EC31F0E0ECFD
:1061D00031F01F0E366F18EC32F00B35D8B0C8EC2A
:1061E00031F0D8A00335D8B01200362FEBEF30F0E5
:1061F00034B1EFEC31F012000101346B04510511A0
:10620000061107110008D8A0ECEC31F0D8A002EC80
:1062100032F0D8B01200086B096B0A6B0B6B18ECEC
:1062200032F01F0E366F18EC32F007510B5DD8A418
:1062300026EF31F006510A5DD8A426EF31F0055162
:10624000095DD8A426EF31F00451085DD8A039EFDC
:1062500031F00451085F0551D8A0053D095F065192
:10626000D8A0063D0A5F0751D8A0073D0B5FD89024
:106270000081362F13EF31F034B1EFEC31F0346B95
:10628000ECEC31F0D8901CEC32F007510B5DD8A447
:1062900056EF31F006510A5DD8A456EF31F00551A2
:1062A000095DD8A456EF31F00451085DD8A065EF20
:1062B00031F0003F65EF31F0013F65EF31F0023F13
:1062C00065EF31F0032BD8B4120034B1EFEC31F0AC
:1062D00012000101346BECEC31F0D8B0120021EC6B
:1062E00032F0200E366F003701370237033711EED8
:1062F00033F00A0E376FE7360A0EE75CD8B0E76E68
:10630000E552372F7BEF31F0362F73EF31F034B198
:106310002981D890120021EC32F0200E366F003720
:1063200001370237033711EE33F00A0E376FE736C5
:106330000A0EE75CD8B0E76EE552372F97EF31F0E1
:10634000362F8FEF31F0D890120001010A0E346F12
:10635000200E366F11EE29F03451376F0A0ED890A7
:10636000E652D8B0E726E732372FB0EF31F00333EB
:10637000023301330033362FAAEF31F0E750FF0F1D
:10638000D8A00335D8B0120029B1EFEC31F01200DB
:10639000045100270551D8B0053D01270651D8B05A
:1063A000063D02270751D8B0073D032712000051D0
:1063B000086F0151096F02510A6F03510B6F1200F0
:1063C0000101006B016B026B036B12000101046B96
:1063D000056B066B076B12000335D8A01200035142
:1063E000800B001F011F021F031F003FFFEF31F052
:1063F000013FFFEF31F0023FFFEF31F0032B342B71
:10640000032512000735D8A012000751800B041F86
:10641000051F061F071F043F15EF32F0053F15EF5C
:1064200032F0063F15EF32F0072B342B0725120010
:106430000037013702370337083709370A370B3778
:1064400012000101296B2A6B2B6B2C6B2D6B2E6BB1
:106450002F6B306B316B326B336B120001012A51A1
:106460000F0B2A6F2B510F0B2B6F2C510F0B2C6F17
:106470002D510F0B2D6F2E510F0B2E6F2F510F0B18
:106480002F6F30510F0B306F31510F0B316F325175
:106490000F0B326F33510F0B336F120000C124F119
:1064A00001C125F102C126F103C127F104C100F1A8
:1064B00005C101F106C102F107C103F124C104F1D4
:1064C00025C105F126C106F127C107F1120000011F
:1064D0002550FE0AD8B475EF32F000012550FD0AB0
:1064E000D8B475EF32F0898401D08994000EC76E5C
:1064F000220EC66E050EE82EFED7120000012550B2
:10650000FE0AD8B48CEF32F000012550FD0AD8B451
:106510008CEF32F0899401D08984050EE82EFED7E5
:10652000120067EC32F000012550FD0AD8B4A4EF48
:1065300032F09E96C69E000EC96EFF0E9EB602D029
:10654000E82EFCD7ADEF32F09E96C69E010EC96EC6
:10655000FF0E9EB602D0E82EFCD79E96C69E000E79
:10656000C96EFF0E9EB602D0E82EFCD7C9CFAFF59C
:106570009E96C69E000EC96EFF0E9EB602D0E82EF5
:10658000FCD7C9CFB0F59E96C69E000EC96EFF0E11
:106590009EB602D0E82EFCD7C9CFB1F59E96C69E16
:1065A000000EC96EFF0E9EB602D0E82EFCD7C9CFF2
:1065B000B2F59E96C69E000EC96EFF0E9EB602D024
:1065C000E82EFCD7C9CFB3F59E96C69E000EC96EC5
:1065D000FF0E9EB602D0E82EFCD7C9CFB4F59E962A
:1065E000C69E000EC96EFF0E9EB602D0E82EFCD7E6
:1065F000C9CFB5F57EEC32F0120067EC32F0000145
:106600002550FD0AD8B410EF33F09E96C69E800E3A
:10661000C96EFF0E9EB602D0E82EFCD719EF33F0FC
:106620009E96C69E810EC96EFF0E9EB602D0E82EC3
:10663000FCD79E96C69EAFC5C9FFFF0E9EB602D080
:10664000E82EFCD79E96C69EB0C5C9FFFF0E9EB62B
:1066500002D0E82EFCD79E96C69EB1C5C9FFFF0E9C
:106660009EB602D0E82EFCD79E96C69EB2C5C9FF44
:10667000FF0E9EB602D0E82EFCD79E96C69EB3C5EE
:10668000C9FFFF0E9EB602D0E82EFCD79E96C69E8E
:10669000B4C5C9FFFF0E9EB602D0E82EFCD79E9669
:1066A000C69EB5C5C9FFFF0E9EB602D0E82EFCD728
:1066B0007EEC32F0120067EC32F000012550FD0A4A
:1066C000D8B46EEF33F09E96C69E070EC96EFF0ECD
:1066D0009EB602D0E82EFCD777EF33F09E96C69E8A
:1066E000090EC96EFF0E9EB602D0E82EFCD79E960C
:1066F000C69E000EC96EFF0E9EB602D0E82EFCD7D5
:10670000C9CFAFF59E96C69E000EC96EFF0E9EB60F
:1067100002D0E82EFCD7C9CFB0F59E96C69E000EDB
:10672000C96EFF0E9EB602D0E82EFCD7C9CFB1F5D8
:106730009E96C69E000EC96EFF0E9EB602D0E82E33
:10674000FCD7C9CFB2F57EEC32F067EC32F09E9602
:10675000C69E26C0C9FFFF0E9EB602D0E82EFCD70B
:106760009E96C69E000EC96EFF0E9EB602D0E82E03
:10677000FCD7C9CFB6F57EEC32F0120067EC32F0F0
:1067800000012550FD0AD8B4D1EF33F09E96C69E85
:10679000870EC96EFF0E9EB602D0E82EFCD7DAEF48
:1067A00033F09E96C69E890EC96EFF0E9EB602D02D
:1067B000E82EFCD79E96C69E000EC96EFF0E9EB6B2
:1067C00002D0E82EFCD79E96C69E800EC96EFF0EA4
:1067D0009EB602D0E82EFCD79E96C69E800EC96E4D
:1067E000FF0E9EB602D0E82EFCD79E96C69E800E67
:1067F000C96EFF0E9EB602D0E82EFCD77EEC32F0BA
:10680000120000012550FE0AD8B410EF34F0000148
:106810002550FD0AD8B427EF34F05BEC33F01200BA
:1068200067EC32F09E96C69E8F0EC96EFF0E9EB626
:1068300002D0E82EFCD79E96C69E000EC96EFF0EB3
:106840009EB602D0E82EFCD77EEC32F0120067EC48
:1068500032F09E96C69E8E0EC96EFF0E9EB602D078
:10686000E82EFCD79E96C69E000EC96EFF0E9EB601
:1068700002D0E82EFCD77EEC32F012000001255049
:10688000FE0AD8B477EF34F000012550FD0AD8B4E1
:10689000A4EF34F067EC32F09E96C69E27C0C9FF85
:1068A000FF0E9EB602D0E82EFCD79E96C69E010E25
:1068B000C96EFF0E9EB602D0E82EFCD77EEC32F0F9
:1068C00067EC32F09E96C69E910EC96EFF0E9EB684
:1068D00002D0E82EFCD79E96C69EA50EC96EFF0E6E
:1068E0009EB602D0E82EFCD77EEC32F0120067ECA8
:1068F00032F09E96C69E27C0C9FFFF0E9EB602D0FC
:10690000E82EFCD79E96C69E450EC96EFF0E9EB61B
:1069100002D0E82EFCD77EEC32F067EC32F09E9687
:10692000C69E8F0EC96EFF0E9EB602D0E82EFCD713
:106930009E96C69E000EC96EFF0E9EB602D0E82E31
:10694000FCD77EEC32F0120067EC32F09E96C69EC9
:1069500027C0C9FFFF0E9EB602D0E82EFCD79E9638
:10696000C69E3D0EC96EFF0E9EB602D0E82EFCD725
:106970007EEC32F067EC32F09E96C69E8F0EC96EAA
:10698000FF0E9EB602D0E82EFCD79E96C69EA90E9C
:10699000C96EFF0E9EB602D0E82EFCD77EEC32F018
:1069A000120067EC32F09E96C69E27C0C9FFFF0E0C
:1069B0009EB602D0E82EFCD79E96C69E810EC96E6A
:1069C000FF0E9EB602D0E82EFCD77EEC32F012000D
:1069D00067EC32F09E96C69E27C0C9FFFF0E9EB69A
:1069E00002D0E82EFCD79E96C69E010EC96EFF0E01
:1069F0009EB602D0E82EFCD77EEC32F0120067EC97
:106A000032F09E96C69E910EC96EFF0E9EB602D0C3
:106A1000E82EFCD79E96C69EA50EC96EFF0E9EB6AA
:106A200002D0E82EFCD77EEC32F0120067EC32F098
:106A30009E96C69E910EC96EFF0E9EB602D0E82E9F
:106A4000FCD79E96C69E000EC96EFF0E9EB602D063
:106A5000E82EFCD77EEC32F012000501256B266B88
:106A6000276B286B899A400EC76E200EC66E9E96C5
:106A7000C69E030EC96EFF0E9EB602D0E82EFCD74E
:106A80009E96C69E27C5C9FFFF0E9EB602D0E82E71
:106A9000FCD79E96C69E26C5C9FFFF0E9EB602D0A5
:106AA000E82EFCD79E96C69E25C5C9FFFF0E9EB652
:106AB00002D0E82EFCD79E96C69EC952FF0E9EB607
:106AC00002D0E82EFCD7898A0F01C950FF0A01E1E4
:106AD000120005012E51130A05E005012E51170A77
:106AE0000CE012000501F00E256FFF0E266F0F0E51
:106AF000276F000E286F86EF35F00501F00E256F29
:106B0000FF0E266FFF0E276F000E286F899A400E2A
:106B1000C76E200EC66E9E96C69E030EC96EFF0EF1
:106B20009EB602D0E82EFCD79E96C69E27C5C9FF0A
:106B3000FF0E9EB602D0E82EFCD79E96C69E26C5B6
:106B4000C9FFFF0E9EB602D0E82EFCD79E96C69EC9
:106B500025C5C9FFFF0E9EB602D0E82EFCD79E9633
:106B6000C69EC952FF0E9EB602D0E82EFCD7898A77
:106B70000F01C950FF0A1DE005012E51130A05E05F
:106B800005012E51170A0BE012000501000E256FBA
:106B9000000E266F100E276F000E286F12000501E1
:106BA000000E256F000E266F000E276F010E286F56
:106BB00012000501256B266B276B286B05012E51F2
:106BC000130A05E005012E51170A0CE01200050119
:106BD000000E216F000E226F080E236F000E246F2F
:106BE000FBEF35F00501000E216F000E226F800EC5
:106BF000236F000E246F21C500F122C501F123C5CA
:106C000002F124C503F125C504F126C505F127C508
:106C100006F128C507F11CEC2FF000C125F501C1D4
:106C200026F502C127F503C128F5899A400EC76EE3
:106C3000200EC66E9E96C69E030EC96EFF0E9EB6B1
:106C400002D0E82EFCD79E96C69E27C5C9FFFF0E30
:106C50009EB602D0E82EFCD79E96C69E26C5C9FFDA
:106C6000FF0E9EB602D0E82EFCD79E96C69E25C586
:106C7000C9FFFF0E9EB602D0E82EFCD79E96C69E98
:106C8000C952FF0E9EB602D0E82EFCD7898AC950A1
:106C9000FF0A08E104C125F505C126F506C127F55F
:106CA00007C128F5D890050124332333223321333B
:106CB0002151F00B216F0501216766EF36F0226745
:106CC00066EF36F0236766EF36F02467FBEF35F0AA
:106CD0000501100E2527E86A2623E86A2723E86ABB
:106CE00028231200E86A05012E51130A06E0050167
:106CF0002E51170A0BE0020E120005012851000A5E
:106D000003E12751F00B07E0010E120005012851A5
:106D1000000A01E0010E120029C500F12AC501F1A7
:106D20002BC502F12CC503F125C504F126C505F1DB
:106D300027C506F128C507F1CBEC30F003BF1200E0
:106D400072EC36F0D8A404EF37F0899A400EC76E83
:106D5000200EC66E9E96C69E060EC96EFF0E9EB68D
:106D600002D0E82EFCD7898A899A9E96C69E020E8A
:106D7000C96EFF0E9EB602D0E82EFCD79E96C69E28
:106D800027C5C9FFFF0E9EB602D0E82EFCD79E96FF
:106D9000C69E26C5C9FFFF0E9EB602D0E82EFCD7C0
:106DA0009E96C69E25C5C9FFFF0E9EB602D0E82E50
:106DB000FCD79E96C69E000EC96EFF0E9EB602D0F0
:106DC000E82EFCD7898A899A9E96C69E050EC96EC2
:106DD000FF0E9EB602D0E82EFCD79E96C69EC952E4
:106DE000FF0E9EB602D0E82EFCD7C9B0EDEF36F00C
:106DF000898A0501100E2527E86A2623E86A2723D9
:106E0000E86A28238CEF36F01200899A400EC76E8C
:106E1000200EC66E9E96C69E060EC96EFF0E9EB6CC
:106E200002D0E82EFCD7898A899A9E96C69EC70E04
:106E3000C96EFF0E9EB602D0E82EFCD7898A0501E6
:106E4000256B266B276B286B1200899A400EC76E44
:106E5000200EC66E9E96C69E050EC96EFF0E9EB68D
:106E600002D0E82EFCD79E96C69EC952FF0E9EB653
:106E700002D0E82EFCD7C9CF37F5898A1200899A4B
:106E8000400EC76E200EC66E9E96C69EB90EC96E87
:106E9000FF0E9EB602D0E82EFCD7898A1200899A8E
:106EA000400EC76E200EC66E9E96C69EAB0EC96E75
:106EB000FF0E9EB602D0E82EFCD7898AFF0EE82E80
:106EC000FED7120072EC36F0D8A41200899A400E58
:106ED000C76E200EC66E9E96C69E030EC96EFF0E2E
:106EE0009EB602D0E82EFCD79E96C69E27C5C9FF47
:106EF000FF0E9EB602D0E82EFCD79E96C69E26C5F3
:106F0000C9FFFF0E9EB602D0E82EFCD79E96C69E05
:106F100025C5C9FFFF0E9EB602D0E82EFCD79E966F
:106F2000C69EC952FF0E9EB602D0E82EFCD7898AB3
:106F30000F01C950FF0AD8A4E1EF38F00501FE0E99
:106F4000376F0501FF0E536FFF0E546FFF0E556F25
:106F5000FF0E566F15A63799158691EC32F0AFC526
:106F600038F5B0C539F5B1C53AF5B2C53BF5B3C58D
:106F70003CF5B4C53DF5B5C53EF50784BAC166F12B
:106F8000BBC167F1BCC168F1BDC169F14BC14FF133
:106F90004CC150F14DC151F14EC152F157C159F19F
:106FA00058C15AF100011650010AD8B4E6EF37F083
:106FB00000011650020AD8B40BEF38F00001165049
:106FC000040AD8B430EF38F0E1EF38F00501476B30
:106FD000486B496B4A6B05014B6B4C6B4D6B4E6BB1
:106FE00005014F6B506B516B526B8BA0379B8EEC36
:106FF00022F000C1DAF101C1DBF102C1DCF103C111
:10700000DDF100C13FF501C140F502C141F503C109
:1070100042F54FEF38F00501476B486B496B4A6BFF
:1070200005014B6B4C6B4D6B4E6B05014F6B506B01
:10703000516B526B8EEC22F000C1DAF101C1DBF131
:1070400002C1DCF103C1DDF18BEC23F000C147F597
:1070500001C148F502C149F503C14AF5E1EF38F035
:10706000379BDAC13FF5DBC140F5DCC141F5DDC13D
:1070700042F58EEC22F000C14BF501C14CF502C186
:107080004DF503C14EF58BEC23F000C14FF501C166
:1070900050F502C151F503C152F54FEF38F005012B
:1070A00061675AEF38F062675AEF38F063675AEF5A
:1070B00038F064675EEF38F073EF38F0DAC100F152
:1070C000DBC101F1DCC102F1DDC103F161C504F1F5
:1070D00062C505F163C506F164C507F1CBEC30F07C
:1070E00003BFE1EF38F059C143F55AC144F5B9C5C2
:1070F00045F50501110E326F899A400EC76E200EBC
:10710000C66E9E96C69E060EC96EFF0E9EB602D035
:10711000E82EFCD7898A899A9E96C69E020EC96E71
:10712000FF0E9EB602D0E82EFCD79E96C69E27C5BF
:10713000C9FFFF0E9EB602D0E82EFCD79E96C69ED3
:1071400026C5C9FFFF0E9EB602D0E82EFCD79E963C
:10715000C69E25C5C9FFFF0E9EB602D0E82EFCD7FD
:1071600025EE37F0322F02D0C1EF38F09E96C69E42
:10717000DECFC9FFFF0E9EB602D0E82EFCD7B2EFDD
:1071800038F0898A899A9E96C69E050EC96EFF0EB2
:107190009EB602D0E82EFCD79E96C69EC952FF0E20
:1071A0009EB602D0E82EFCD7C9B0CCEF38F0898A61
:1071B0000501100E2527E86A2623E86A2723E86AD6
:1071C000282315900794120021C500F122C501F172
:1071D00023C502F124C503F1899A400EC76E200E23
:1071E000C66E9E96C69E0B0EC96EFF0E9EB602D050
:1071F000E82EFCD79E96C69E02C1C9FFFF0E9EB622
:1072000002D0E82EFCD79E96C69E01C1C9FFFF0E94
:107210009EB602D0E82EFCD79E96C69E00C1C9FF3E
:10722000FF0E9EB602D0E82EFCD79E96C69EC9528F
:10723000FF0E9EB602D0E82EFCD725EE37F00501F2
:10724000100E326F9E96C69EC952FF0E9EB602D099
:10725000E82EFCD7C9CFDEFF322F22EF39F0898A22
:107260001200899A400EC76E200EC66E9E96C69E6C
:10727000900EC96EFF0E9EB602D0E82EFCD79E96E9
:10728000C69E000EC96EFF0E9EB602D0E82EFCD739
:107290009E96C69E000EC96EFF0E9EB602D0E82EC8
:1072A000FCD79E96C69E000EC96EFF0E9EB602D0FB
:1072B000E82EFCD79E96C69EC952FF0E9EB602D0FF
:1072C000E82EFCD7C9CF2DF59E96C69EC952FF0E5B
:1072D0009EB602D0E82EFCD7C9CF2EF5898A1200BF
:1072E00091EC32F005012F51010A61E005012F51A7
:1072F000020A16E005012F51030A1BE005012F5178
:10730000040A26E005012F51050A2DE005012F5141
:10731000060A3BE005012F51070A41E0D7EF39F09B
:1073200015B01200602FD5EF39F05FC560F5D7EFCB
:1073300039F0B0C500F101010F0E00170101005135
:10734000000A35E001010051050A31E0D5EF39F0BE
:10735000B0C500F101010F0E001701010051000A34
:1073600026E0D5EF39F00501B051000A20E0050113
:10737000B051150A1CE00501B051300A18E00501B2
:10738000B051450A14E0D5EF39F00501B051000ABB
:107390000EE00501B051300A0AE0D5EF39F00501E1
:1073A000B051000A04E0D5EF39F0159012001580B5
:1073B00012008B9097EC2FF0B9C5E8FFD70802E3D5
:1073C00097EC2FF0B9C5E8FFC80802E397EC2FF05F
:1073D000B9C5E8FFB90802E397EC2FF0B9C5E8FF9B
:1073E000AA0802E397EC2FF0B9C5E8FF9B0802E377
:1073F00097EC2FF03FEC37F0F29CF29E8B94C69AFC
:10740000C2909482948C720ED36ED3A4FED78996C8
:107410008A909390F29AF2949D909E909D929E9263
:10742000F298F29201EC34F0FF0EE8CF00F0E82E73
:10743000FED7002EFCD7F290F2868150FF0EE82E88
:10744000FED7F29081A827EF3AF0F29E0300700E6B
:10745000D36EF296F29015840380B8EC2FF09AEF79
:027460000BF02F
:10BF0000E844F926000C160C2B0C3F0C520C640C68
:10BF1000760C860C960CA50CB30CC10CCF0CDC0C6B
:06BF2000E80CF40C000C1B
:0200000400F00A
:0100C800FD3A
:00000001FF
